:2000000020140020E9000000F1000000F300000000000000000000000000000000000000BF
:20002000000000000000000000000000FB0000000000000000000000FF00000001010000C4
:20004000030100000501000007010000090100000B0100000D0100000F0100001101000048
:20006000130100001501000017010000190100001B0100001D0100001F01000021010000A8
:20008000230100002501000027010000290100002B0100002D0100002F0100003101000008
:2000A000330100003501000037010000390100003B0100003D0100003F0100004101000068
:2000C000EF3BE8FF03B40148019001BD01FF00200448854600F070F800480047410700005A
:2000E000C046C046201400201648804716480047FEE7FEE7FEE7FEE7FEE7FEE7FEE7FEE7AE
:20010000FEE7FEE7FEE7FEE7FEE7FEE7FEE7FEE7FEE7FEE7FEE7FEE7FEE7FEE7FEE7FEE78F
:20012000FEE7FEE7FEE7FEE7FEE7FEE7FEE7FEE7FEE7FEE7FEE7FEE7FEE7FEE7FEE7FEE76F
:20014000FEE70000FD040000D100000030B50B46014600202022012409E00D46D5409D42B4
:2001600005D31D469540491B2546954040191546521E002DF1DC30BDD2B201E00270401C8D
:20018000491EFBD270470022F6E710B513460A4604461946FFF7F0FF204610BD30B5044617
:2001A0000020034600E05B1C934203D2E05CCD5C401BF8D030BD0000064C0125064E05E0AF
:2001C000E36807CC2B430C3C98471034B442F7D3FFF782FFC00B0000F00B0000F8B5044634
:2001E0000D460020002C00D100BF002A00D100BF012C01D141263043012A01D11226304395
:20020000022C01D1C0263043022A01D130263043134E307076788027BE43114F7E70012CAC
:2002200008D1FF2100BF0E4EB3781E460E4033468B42F8D10A4E76784027BE43084F7E70CB
:20024000012A0BD10026009603E000BF009E761C0096FF276937009EBE42F6D9F8BD00008B
:200260000004024070B5034614460020002B01D1C0B202E005468035E8B2012902D1051D46
:20028000E8B206E0022903D105460835E8B200E0C0B2012C02D1851CE8B200E0C0B2084D89
:2002A000A870AD7801263543054EB570002201E000BF521C7D252D01AA42F9D970BD0000FF
:2002C000000C024070B500242448007920210840002801D0224D3FE000F046F805462148B0
:2002E000007880210840002836D01E4880780840002801D01A4D02E000F036F805461948BD
:2003000080780007840F022C01DBAD0804E0012C01D16D0800E000BF124880788007C00FED
:20032000002801D02D0101E00C2045430D4800784007840F002C02D1601CC4B207E0032C53
:2003400003D1601C4006040E01E06006040E21462846FFF7FBFE0546284670BD00040240AC
:2003600000127A00000C024000B5C0229178F82211401C4A12781143EA2923D00ADC0A4618
:20038000E03A130000F00AF90A181C20242A2A2A2A161A2AED291FD004DCEB2916D0EC29C5
:2003A0001CD117E0F02903D0F82917D10E4817E00E4815E00E4813E00E4811E00E480FE0F7
:2003C0000E480DE00E480BE00E4809E00E4807E00E4805E00E4803E00E4801E00D4800BF5E
:2003E00000BF00BD201C02400090D003006CDC020048E80100366E010024F400001BB70096
:2004000000127A00808D5B0000093D00C0C62D0080841E0040420F00014610200D4AD0603E
:20042000F120106255205060AA2090600020C043086000BF07480068C007C00F0028F9D0D2
:200440000448006801221043024A10600020D06010627047000002400246F1200B4B1862D2
:20046000AA20586055209860116000BF07480068C007C00F0028F9D00448006801231843EC
:20048000024B186000201862704700000000024010B501231A4600211846FFF79FFE012286
:2004A00011461046FFF7DEFEFFF70CFE034800F023F902480249086010BD00000090D00339
:2004C0001C00002010B500F063F810BD1A20084908722B2048723C2088724D20C8727F205D
:2004E000044909680860AC20034948707047000000040240180000200010024010B580201A
:200500001B4948711A201A49203908722B2048723C2088724D20C872002016494860FFF72F
:20052000D1FE154908600020C0431449086014490860144814490860114903221202891824
:2005400048600F49891888600D498918C8600C49891808610A49891848610949891888611B
:2005600007498918C861AC200849487010BD00002004024000B001401C00002080E200E0EA
:2005800000E100E0C0C0C0C000E400E000100240AC200149487070470010024030B474460F
:2005A000641E2578641CAB4204D3635D5B00E31830BC18471D46F8E702E008C8121F08C189
:2005C000002AFAD170477047002001E001C1121F002AFBD170470000F8B50446606800F068
:2005E0005BF80646A06800F057F8074600F066F80025ED4309E0307868400006800D0B4905
:200600000858290A48400546761C38467F1E0028F1D1ED43206800F03FF8A84201D0012022
:2006200000E0002000900098F8BD00002000002070B5002561246402202221461548FFF76C
:20064000ADFD002823D120222146403111484030FFF7A4FD00281AD12022A1180D482030A7
:20066000FFF79CFD002812D120222146603109486030FFF793FD002809D1102221468031F3
:2006800004488030FFF78AFD002800D100E00125284670BD300B0000014600200A06FF2373
:2006A0001B020B401B021A43FF231B040B401B0A1A430B0E1A4310467047000010B50021E1
:2006C00013E0084608220AE0C307DB0F002B04D04308074C6340184600E04008521E002AB1
:2006E000F2D18B00034CE050491CFF29E9D910BD2083B8ED2000002010B5044603492046C8
:20070000FFF724FD0249087010BD000040420F000400002070B505460E4672B62C460BE034
:200720002046FFF779FEA004800C002801D1FFF7C9FE012080022418B442F1D362B670BD21
:2007400010B5012464072E482E4908602E482F4908602F482F4908602A4800680068401CA4
:2007600000283CD0274800680068284909680968884234D027480068406800282FD12149D4
:2007800009688868FFF788FF6114401803218903884224D2FFF74CFF002820D1194800681B
:2007A000FFF71AFF00281AD1FFF790FEFFF770FE00F036F8144800F0B2F80C22114801682B
:2007C000114800F077F800BFBFF34F8F12481349C860BFF34F8F00BF00BF00BFFDE772B65B
:2007E000012109042046FFF7CEFC01210903086880F3088800BF48688047002010BD0000E0
:2008000020C000000C000020001450001000002000105000140000200400FA0500ED00E0D4
:20082000F0B5FFB0FFB083B0214909684868FFF733FF00900321890301200003FFF76AFF0C
:2008400001273F031A4909688868FFF725FF8505AD0D174909688868FFF71EFF8005800D26
:20086000002800D06D1C00261CE0FF220121890201A8FFF781FC002406E0B002011900987D
:20088000415C01AA1155641C012080028442F4D3024601A9384600F00DF8012080023F189B
:2008A000761C6D1E002DE0D17FB07FB003B0F0BD0C000020F8B505460E461746009672B6EC
:2008C000002407E0A2089300009AD1582819FFF7C3FD241DBC42F5D3FFF7F4FD62B6F8BD5B
:2008E000014672B608208F4AD060F120106255205060AA2090600020C043086000BF8948DB
:200900000068C007C00F0028F9D00120854A10600020D060F020106262B600207047014680
:2009200072B610207F4AD060F120106255205060AA2090600020C043086000BF7948006891
:20094000C007C00F0028F9D00120764A10600020D060F02010621046006804221040002891
:2009600005D004206F4A106062B60120704762B60020FBE770B503461D46F120694E306220
:20098000002415E072B6AA20664E70605520B06010782870521C6D1C62B600BF6148006844
:2009A000C007C00F0028F9D001205E4E3060641C8C42E7D3F0205B4E3062002070BDF7B507
:2009C000FFB0FFB089B006460F460021FFA8C161012104914802874206D9FFA8C161C0695A
:2009E0007FB07FB00CB0F0BD029600240DE002980078FFA988610298401C02908869FF2844
:200A000001D000200490601C84B2BC42EFD30498002809D0444845490860FFA83946826AAE
:200A20003046FFF7A7FF6DE0750AF119681C4002814202D90120039001E000200390710AA7
:200A400049020191F105C90D0091039800280FD0002408E00198007805A908550198411C9C
:200A60000191601C84B2012080028442F2DB0EE0002408E00198007805A908550198411CF0
:200A80000191601C84B2012040028442F2DB00240DE0FFA8806A01780098001905AA11543C
:200AA000FFA8806A411CFFA88162601C84B2BC42EFD30398002816D01B481C490860680209
:200AC000FFF72DFF184819490860691C4802FFF726FF154815490860680205AA01218902F7
:200AE000FFF748FF0EE01048104908606802FFF716FF0D480D490860680205AA01214902A4
:200B0000FFF738FFFFA8C0696AE730B50446002304E025781570641C521C5B1C8B42F8D332
:200B200030BD000000000240CDAB341208000020484A5F3735305F544654000000000000C6
:200B400000000000000000000000000000000000484A59422D373530305446540000000081
:200B6000000000000000000000000000000000004241543332413237394B4D3634464200CC
:200B80000000000000000000000000000000000043414E5F5354445F4348305F3530304BE0
:200BA000627073000000000000000000000000008907000081070000DF07000000000000F2
:200BC000F00B00000000002020000000B8050000100C000000FF002024000000B805000001
:200BE000100C00002000002000140000C805000000000000000000000000000000000000B8
:200C00000000000000000000C00000000000000001200649087000BF0448007880210840C0
:140C20000028F9D00120024908707047000C024000000020C6
:2010000090570020E9100000F1100000F310000000000000000000000000000000000000CC
:20102000000000000000000000000000FB1000000000000000000000FF100000015D000038
:2010400051400000B5400000FD400000454100008D410000D54100001D420000654200005D
:20106000AD420000F5420000414300008D430000A1430000ED430000014400001544000044
:2010800061440000C5440000314500009D450000094600007546000089460000D546000056
:2010A0002147000069470000B5470000214800003548000049480000B5480000214900003E
:2010C000EF3BE8FF03B40148019001BD01FF00200448854600F094F900480047A982000042
:2010E000C046C046905700201648804716480047FEE7FEE7FEE7FEE7FEE7FEE7FEE7FEE7EB
:20110000FEE7FEE7FEE7FEE7FEE7FEE7FEE7FEE7FEE7FEE7FEE7FEE7FEE7FEE7FEE7FEE77F
:20112000FEE7FEE7FEE7FEE7FEE7FEE7FEE7FEE7FEE7FEE7FEE7FEE7FEE7FEE7FEE7FEE75F
:20114000FEE7000045600000D110000030B50B46014600202022012409E00D46D5409D42F0
:2011600005D31D469540491B2546954040191546521E002DF1DC30BD70B5002425460028D4
:2011800001DA01244042002901DA01254942FFF7DDFFAC4200D04042002C00D0494270BD52
:2011A00003460B439B0703D009E008C9121F08C0042AFAD203E00B780370401C491C521E6C
:2011C000F9D27047D2B201E00270401C491EFBD270470022F6E710B513460A460446194659
:2011E000FFF7F0FF204610BD30B504460020034600E05B1C934203D2E05CCD5C401BF8D0B6
:2012000030BD0321001D401E037812021A43491EF9D510467047034603220870000A491CBF
:20122000521EFAD518467047024670B54A40D30FDB0740002DD04A002AD0010E140E0002EB
:2012400012020919400A520A8418E50104465443000A120A2E045043A4194219200CC54318
:20126000AA18120C0125AD03521C521912047F39240400D0521C104301D44000491EC2B268
:201280000C06C0092018401C4008802A02D003E0002070BD40084000002900DA00201843E5
:2012A00070BD70B502464A40D50F40004A00ED0740085208002814D0002A12D0C40DD30D3D
:2012C00041020120C0055202490A520AE41A091812187D34914201D3641C00E04900002C6C
:2012E00001DA002070BD0023914201D3891A0343400849000028F7D100290AD0914202D1E9
:201300000121C90705E0914201D2012101E00121C943E005C018401900F030F870BD10B5FF
:2013200000229623114600F031F810BDC20FD207400040080BD0C10D0723DB01C918400291
:201340000905400A1143C20840071143704700200146704710B5002904DB0124E407404248
:201360008C412146002B04DB1C460123DB075242A341994200D1904210BD0000002904DAFD
:20138000401C490001D140084000704770B40024050C05D11024000402D1002921D011240E
:2013A000050E01D100020834050F01D10001241D850F01D18000A41C002801DB4000641C78
:2013C000002908D020252E1B0D46F540A14000D001212943084301061B1B000ADB1D02D556
:2013E000002070BC7047DB05181880180029F8DA401C4900F5D170BC400840007047000071
:20140000064C0125064E05E0E36807CC2B430C3C98471034B442F7D3FFF75EFE808C000006
:20142000B08C000070B58C180578401C6B075B0F01D10378401C2A1106D10278401C03E07E
:2014400006780E70401C491C5B1EF9D12B0705D40023521E0DD40B70491CFAE70378401C75
:20146000CB1A921C03E01D780D70491C5B1C521EF9D5A142D8D3002070BD0000F0B591B009
:20148000032080031B4908600121C9042320400302F092F8312005F0FDFA232676031D27A6
:2014A000FF01002522E0FF22402101A8FFF78AFE002407E0A80100190E490968085C01A9B9
:2014C0000855641C402CF5D301AA4021304606F0F5FF40366D1C7F1E4B2109012846FFF719
:2014E00035FE002902D1312005F0D4FA002FDAD111B0F0BD9C020020F0B591B02320400337
:201500001449086001460320800302F055F80325AD031D26F601002718E0FF22402101A87E
:20152000FFF750FE002407E0B801001909490968085C01A90855641C402CF5D301AA40219C
:20154000284606F0BBFF40357F1C761E002EE4D111B0F0BD9C02002010B5002100BF0EE027
:201560004A00204B9A5A204B9A4206D24A001D4B9A5A12184B001B4CE2524A1CD1B20329D8
:20158000EEDB1A4A1268322A04D2184A12681218164B1A60164A1268164B1B689A4204D221
:2015A000134A12681218124B1A60134A1268134B9A4204D2104A126812180F4B1A60104A40
:2015C0001278002A0AD10F4A12880F4B9A4208D20C4A128812180B4B1A8002E00022094B17
:2015E0001A8010BD1C00002010270000380000203000002034000020040000208813000056
:201600003C0000203E000020B80B000010B502469000074BC018405C002802D00320C043CA
:2016200010BD01209300024C1B1958540020F7E72016002010B509490B680968491C074CF4
:2016400021600749C8542146096801221203914202D300212246116010BD000000000020FE
:20166000EC020020F0B589B006A908A802F08CFA0546089803906D480468089906988842FF
:201680007ED208988442FBD2C8E00698A04203D30698001B079004E00898001B06994018E3
:2016A00007900398002803D00398401E039000E0B8E0285DEB2871D10898401E611C08405C
:2016C000285C9028F7D10798062868D90898401EA11C08402E5C36020898401EE11C0840F0
:2016E000285C06430898401E211D0840285C05900598000205900898401E611D0840285C04
:201700000599084305900598C04380B2B0425DD1089886425AD80798B04256D30898401E07
:20172000A11D08402F5C3F020898401EE11D0840285C07433F020898401E491C0840285C55
:2017400007433F020898401E491C0840285C07430020C04332460A3A00900898401E491CB3
:201760000840029001462846089B00F031FC04900498B84214D1089883B230460A3800E09E
:2017800051E082B20898401E21460A31084080B201460290284603F023FA06E02FE02DE071
:2017A00023480068401C224908600020285500220898401E611C08402A54A0190899491E66
:2017C000084004461948046028E02BE019480068401C184908600020285500220898401EF4
:2017E000611C08402A540898401E10490968491C08400E490860084604680FE012E0079838
:2018000002280AD30898401E08490968491C0840064908600846046800E003E006988442BC
:2018200000D032E700BF09B0F0BD0000E0020020B0020020B402002070B5014600205825E7
:201840006D5A1C2635402B4658256B5204251D40002D04D008251D40002D00D00120042507
:201860001D40002D2DD053256D5C10263540002D27D01A4DA94201D1194A00E0194A0024E3
:201880000CE001E00125D581D589ED07ED0F002DF8D10225D5811032651CECB2102CF0DBD6
:2018A000FF2650256E5252256D5C002D02D0002652256E540126F60350256E52FF26073679
:2018C0006E5208251D40002D06D052256D5C002D02D0002652256E5470BD00000054044058
:2018E0000055044000590440582211527047014600205322525C10231A40002A08D0532290
:20190000525C0C231A409210032A18D1032016E05422525A0123DB031A40002A0ED05322C4
:20192000525C0C231A409210032A05D05322525C9207920F032A01D1022000E00120704796
:201940000246002058239B5A0B40002B01D0012000E00020704710B5002A0AD056231B5AD9
:201960000C0223435624235256231B5A8B43235209E056231B5A0C02A343562423525623A0
:201980001B5A0B43235210BDF8B504460D46012700263448844203D10121022000F01EFA48
:2019A0002878401EA0702088FF210131084320802088400840002080A878401EC1B25A20F9
:2019C000015568790007000CE97909020843A97908435C210853288981B240200153A86818
:2019E000C000C10C42200153A88981B244200153E868C000C10C46200153288A81B24820A4
:201A000001532869C000C10C4A200153A88A81B24C2001536869C000C10C4E2001535020E1
:201A2000005B297909020843502108535020005B297988435021085300E0761C5020005B46
:201A40004007400F2979884202D007488642F4D15020005B4007400F2979884200D0002712
:201A60003846F8BD00540440FFFF00000146144AC889C007C00F00280AD00120C88100E0C5
:201A8000521EC889C007C00F002801D0002AF7D1C889C007C00F00280FD10220C881042086
:201AA000C881487A400840004872487A38239843487200204872012070470020FCE7000072
:201AC000FFFF00000246507A012318435072507A0B78DB0018435072087A012808D18888DC
:201AE00050814868000C0123DB031843908108E0087A002805D1508148688000204B1840BF
:201B00009081487A012804D1507A40231843507206E0487A002803D1507A4023984350723C
:201B2000087D002804D0507A80231843507203E0507A8023984350720878002811D1C87AE1
:201B40001072087B1070487B5070887B9070CB7BD370087C10714B7C5371887C9071CB7C15
:201B6000D371887A002803D00120C002D08101E00820D081FF200130D0810120704700001D
:201B8000FC1F0000002904D0427A80231A43427203E0427A80239A434272704730B5024606
:201BA00000200F4B5024A45A0D022C435025AC525024A45A8C43AC5200E05B1E5024A45A3E
:201BC0006407640F8C4201D0002BF6D15024A45A6407640F002C01D0002000E0012030BD3B
:201BE000FFFF0000F0B587B006460C460027002006906020875BF807C00F002802D0012144
:201C00006020815355E0FF20000238400005000F06902B48864204D106980001294945187A
:201C200006E02948864203D106980001274945180420E881A8890121C9030840002809D050
:201C4000012069460872A889C004C00869890843019007E0002069460872A8891C490840A1
:201C600080100190287A6946C872002003E02A5C03A90A54401C6946C97A8142F7DCA08819
:201C8000172801DB0020A08061881822514322460832881818226946FFF782FA6188481C48
:201CA0001721FFF769FA6180A088401CA0806020875B022038400028A5D007B0F0BD000011
:201CC00000540440005504400058044000590440FC1F000010B502461D4BD089C007C00F1B
:201CE00000280AD00120D08100E05B1ED089C007C00F002801D0002BF7D1D089C007C00F4D
:201D0000002801D0002010BD507A012420435072507A3824A0435072C87A1072487A002850
:201D20000FD1087B1070487B5070887B9070CC7BD470087C10714C7C5471887C9071CC7CD0
:201D4000D471FF200130D0814000D081107ADAE7FFFF0000F8B504460D460020002C00D15C
:201D600000BF002A00D100BF012C01D141263043012A01D112263043022C01D1C026304310
:201D8000022A01D130263043134E307076788027BE43114F7E70012C08D1FF2100BF0E4E56
:201DA000B3781E460E4033468B42F8D10A4E76784027BE43084F7E70012A0BD10026009681
:201DC00003E000BF009E761C0096FF276937009EBE42F6D9F8BD000000040240002905D06F
:201DE000054A12780243044B1A7004E0024A12788243014B1A70704720040240002905D07C
:201E0000054AD27E0243044BDA7604E0024AD27E8243014BDA7670470008024070B50346EF
:201E200014460020002B01D1C0B202E005468035E8B2012902D1051DE8B206E0022903D19F
:201E400005460835E8B200E0C0B2012C02D1851CE8B200E0C0B2084DA870AD780126354350
:201E6000054EB570002201E000BF521C7D252D01AA42F9D970BD0000000C024070B5002468
:201E80002448007920210840002801D0224D3FE000F046F8054621480078802108400028E2
:201EA00036D01E4880780840002801D01A4D02E000F036F80546194880780007840F022CAA
:201EC00001DBAD0804E0012C01D16D0800E000BF124880788007C00F002801D02D0101E0CA
:201EE0000C2045430D4800784007840F002C02D1601CC4B207E0032C03D1601C4006040ED8
:201F000001E06006040E21462846FFF71FF90546284670BD0004024000127A00000C02407F
:201F200000B5C0229178F82211401C4A12781143EA2923D00ADC0A46E03A130006F09AF861
:201F40000A181C20242A2A2A2A161A2AED291FD004DCEB2916D0EC291CD117E0F02903D039
:201F6000F82917D10E4817E00E4815E00E4813E00E4811E00E480FE00E480DE00E480BE067
:201F80000E4809E00E4807E00E4805E00E4803E00E4801E00D4800BF00BF00BD201C02400C
:201FA0000090D003006CDC020048E80100366E010024F400001BB70000127A00808D5B00C0
:201FC00000093D00C0C62D0080841E0040420F00FFB50C460021099800BF16E066185F1EDD
:201FE0003E40009FBE5D3606704000250AE0C60FF607002E04D04600064F7E40304600E02B
:2020000040006D1C082DF2DB491C9142E6DB04B0F0BD0000B71DC10408B501460A78CB7839
:202020001A436B461A704A7852108B785B001A43D3B26A4653708A7892104B789B001A43D2
:20204000D3B26A469370CA78D2100B78DB001A43D3B26A46D370127810066A4652781204C1
:2020600010436A469278120210436A46D278104308BD000010B50446002006F001F9022891
:2020800041D121480078002802D101201E4908701D48007801281FD11B484078401C1A4982
:2020A000487021465A20FFF751F817494978884229D800201449487008468078401C88708D
:2020C000084680780A2803D30020887002200870002006F001F916E00B480078022812D122
:2020E00009484078401C0849487021467D20C000FFF72CF804494978884204D80020024975
:20210000487006F0E9F810BD6400002000B587B0002168460171042141710A4802900146B0
:202120000391049105910848069001A806F0F2F800F05AF800F00CF80021044803F091F951
:2021400007B000BDFFFFFF1FC12100000205000010B51848184948600020087201200870A5
:2021600000204872012088721448FFF77FFC12491248FFF7A7FC01211048FFF703FD0D488A
:202180005E300D4948600020087201200870002048720120887209481030FFF767FC064952
:2021A00006481030FFF78EFC012104481030FFF7E9FC10BD81070000D8130020105504407F
:2021C00010B5044607496068884204D005495E396068884205D1E17A22460C32606800F034
:2021E00063FC10BDDF07000000B587B00E4802900021684601730171417381730821C1733F
:20220000002004E0002204A90A54411CC8B26946C97B8142F6DC0548FFF728FC01A90348D2
:20222000FFF750FC07B000BD890700000055044030B587B00446002520680290A179684652
:20224000C1736179417300210173017100BF05E020460830415D04A841556D1C6846C07B21
:20226000A842F5D8084902984018002808D101A90648FFF72FFD0021029800F09DFB00E026
:2022800000BF00BF07B030BD77F8FFFF00550440FEB504460E460020019005F0AFFF002849
:2022A0004DD103208003844203D023204003844202D1FF34FF34023461204002844202D0AB
:2022C0002148844238D100962048009E864230D2E01FFF38FA380290029800F093F9074603
:2022E0000020C0431A49086025460EE028781849097848400006800D16490858144909686D
:20230000090A4840124908606D1C0098411E00910028EBD10E480068C0430D49086008469D
:202320000068B84202D1002001900AE00120019007E00220019004E00320019001E00420E4
:2023400001900198FEBD000000620400009E0300900200203C88000010B50124640701F0D5
:2023600021FC09480068094988420AD106484068002808D161132046FEF72BFF02F07CFB37
:2023800001E002F04FFB10BD94020020A55A7AA770B590B000261F48008A1E49498A8842FD
:2023A00005DB1C48008A1B49498A401A84B2002C2BD0FF2240216846FEF704FF00250CE028
:2023C0001448418A1430405C694648551148408A401C10494882681C85B2A542F0DB214634
:2023E0000C48143005F0BAFE0A496A460868214606F064F80646002E05D10648006800194D
:202400000449086002E0012600E00026304610B070BD0000381B002010B500202749087055
:2024200001F0C0FB264840682649884204D0244840682549884210D121484068214988425B
:2024400002D101201D49087002202049087005F0B7FD002005F0F8FD2EE0194840681C4978
:20246000884224D100F0A0F81A4880680121C90488421CD21748006861214902884216D1DF
:202480001448416823204003FFF702FF00280ED1FFF732F800F05AF80F4A51681068FFF7D1
:2024A000F7FE002803D105F0CFFD05F039FE05F087FD01200549087010BD00007902002076
:2024C00094020020A33A7AA7A88A7AA777020020A55AA55A9C1B0020901B00200146002055
:2024E0000A06FF231B020B401B021A43FF231B040B401B0A1A430B0E1A4310467047000037
:2025000010B50024312004F0C5FA0E4A51681068FFF7BEFE002812D1FEF7B0FF00F044F8B8
:20252000312004F0B7FA0848416823204003FFF7AFFE002801D1012402E0002400E0012459
:20254000204610BD901B00209C1B002000B5134800F058F8124908601048001D00F052F8E4
:202560000F494860084600686121490288420FD10B4840680B49884202D90020C04304E033
:20258000074840686121490240180549886003E00020C0430249886000BD000004C000002F
:2025A000901B0020003E070000B5124800F02AF8114908600F48001D00F024F80E494860A9
:2025C000084600686121490288420ED10A4840680A49884202D90020C04303E006484068E1
:2025E000074940180449886003E00020C0430249886000BD046004009C1B0020009E030028
:202600000062040030B504460025204603F0FDF805462846FFF762FF0546284630BD0246B4
:202620000020082905D30A2903D80C2A26D1012024E00E2903D8102A20D101201EE012297A
:2026400003D8142A1AD1012018E0162903D8182A14D1012012E01E2903D8202A0ED101209D
:202660000CE02E2903D8302A08D1012006E03E2903D8402A02D1012000E000207047014664
:202680000020022903D3082901D8012010E00C290BD0102909D0142907D0182905D0202969
:2026A00003D0302901D0402901D1022000E00020704710B500F034FF00F00CF900F062FBDF
:2026C00000F002F810BD0000FEB5002455480078912852D100F0F4F80128FAD152480068A9
:2026E0005249086008460079F021884320304F49087108460079000900014A49097A0907DC
:20270000090F0843494908714648807A401E4549887208460189C088401E81422ED2082173
:2027200042484030017100BF0EE03E4841883E48801D415C3D48401D01553A484088401C93
:2027400038494880601CC4B2072CEED33748066840300779002406E03448001D005D6946BE
:202760000855601CC4B2082CF6D3012000F0ECFD6A463946304600F0CFF952E02948018989
:20278000C088401E814242D12648007925498978401AC5B2072D2FDC681CC1B22348403085
:2027A000017100240EE01F4841881F48801D415C1E48401D01551B484088401C19494880FA
:2027C000601CC4B2AC42EEDB1848066840300779002406E01548001D005D69460855601C29
:2027E000C4B2082CF6D3012000F0AEFD6A463946304600F091F914E000F0E2FD0020094956
:20280000087009490868092100F0CAF909E000F0D7FD00200349087003490868092100F03A
:20282000BFF9FEBDD029002068290020382400202049097800293CD01E498978482251435A
:202840001D4A51581D4A116000200CE01949897848225143184A8918091D0A5C1749091D0E
:202860000A54411CC8B21349897848225143124A8918403109798142E8DC0E49897848228F
:2028800051430D4A891840310A790C4940310A7101224A7107490978491E064A1170114639
:2028A0008978491C917011468978082901D3002191707047A423002064210020F0230020BC
:2028C0000349487B012802D10021014A51737047E029002010B533484068002861D1314822
:2028E000007B030005F0C6FB07590512212E3D4A59002D480078002807D000202A49087007
:202900002A490868012100F04BF947E026480078002809D000202449087025498A880123C7
:202920000868891D00F04CF938E01F480078002807D000201C4908701C490868022100F071
:202940002FF92BE018480078002809D000201649087017498A8809230868891D00F030F9A7
:202960001CE011480078002807D000200E4908700E490868092100F013F90FE00A480078F6
:20298000002809D000200849087009498A8803230868891D00F014F900E000BF00BF00F062
:2029A0000FFD10BDE0290020D029002068290020802400207047000070B504460D46364890
:2029C0000068A04267D1002D65D134480078222852D004DC202841D021285AD145E0902828
:2029E00002D0912855D115E02C48C08801280AD100202A49087000F0E3FC29490868002194
:202A000000F0CEF805E0032000F09EFCA020234908703FE021480089401C2049088108461D
:202A20000089C98888420AD100201C49087000F0C7FC1B490868002100F0B2F80DE017488C
:202A4000807A002806D000F0BBFC1449087B00F05BFC02E0032000F077FC1BE0062000F037
:202A600073FC11200D49087014E0062000F06CFC11200A4908700DE000200849087000F0B4
:202A80009FFC08498A8809230868891D00F098F800E000BF00BF70BDA8230020D0290020E7
:202AA000682900208024002070B50346184C2478082C2CD2164C647848256C43154D2B51C9
:202AC00000200AE0155C124C647848267443114EA419241D2554441CE0B28842F2DB0C4C65
:202AE000647848256C430B4D641940342171084C2478641C064D2C702C466478641C6C70FA
:202B00002C466478082C02D30025014C657070BDA423002064210020F0B587B007460D46E2
:202B200016461D480760002406E031781A48001D0155761C601CC4B2AC42F6DB2C4605E04B
:202B4000AA211548001D0155601CC4B2082CF7DB11480068029008216846C17300214173AF
:202B600001730171002406E00B48001D015D04A80155601CC4B2082CF6DB01A90748FFF7AF
:202B8000A9F800210298FFF717FF012102484030017107B0F0BD0000A82300200055044097
:202BA00070B504460D462946204603F08DFF70BD70B504460D462946204603F093FF70BD89
:202BC000F8B504460D4616461F463B4632462946204603F088FFF8BDF0B585B006460F4672
:202BE000154665480078002804D009213046FFF7D7FFBEE0002D01D0602D04D90921304647
:202C0000FFF7CEFFB5E05D4806608580002405E0395D5A48801D0155601C84B2AC42F7DBA6
:202C200000205549487008468580FF2088727F20087308468088082831D20120C880084658
:202C400080884880012008814C4800684C49086008460079F021884349490871084600798C
:202C600000090001444909790907090F08434449087141480079401CC1B241484030017186
:202C8000002407E03D48801D015D3D48401D0155601C84B238488088A042F3DC4CE0072132
:202CA000681CFEF753FA002907D0072128460830FEF74CFA3049C88005E00721681CFEF7FE
:202CC00045FA2D49C88006202B494880012008812A4800682A49086008460079F021884393
:202CE0001030274908710846007900090001224989880905090F08432149087108468088B4
:202D0000FF21090288431C4989880902FF221202114008431A498880082119484030017194
:202D2000002407E01548801D015D1548801D0155601C84B2062CF5D3114800680390104888
:202D4000403000790290002406E00D48001D005D69460855601C84B2082CF6D3012000F053
:202D6000F3FA9020044908706A4602990398FFF7D3FE05B0F0BD0000D02900206829002018
:202D80003824002010B5FFF753FD14484079002823D01248403800790009002806D0012801
:202DA00007D002280AD0032810D10CE000F010FA0FE000F0C5F800F011FB0AE000F010F8CC
:202DC00000F00CFB05E000F06BF902E0FFF7F2FD00BF00BF00210148417110BD3024002021
:202DE00010B55348007811281AD15248006852498842F9D14F4800790007000F4C49097A68
:202E00000907090F88420CD000204949087000F0D7FA4A498A8804230868891DFFF7D0FE53
:202E200084E043480089401C414908810846807A401E887208460089C988884249DA3D4871
:202E400040300079082822D03A48403000790C281DD0384840300079102818D03548403065
:202E60000079142813D033484030007918280ED0304840300079202809D02E484030007957
:202E8000302804D02B484030007940284ED12948403000792649897B884247D100240EE062
:202EA0002448401D015D224842882448801D81541F484088401C1E494880601CC4B21D48C8
:202EC00040300079401EA042EAD8062000F03CFA2CE01748808816494988411A15484030F0
:202EE0000079814222DA00240EE01248401D015D0F4842881148801D8154601CC4B20C4841
:202F00004088401C0A49488009484088084989888842EADB00200649087000F051FA0749F6
:202F20008A8800230868891DFFF74AFE10BD0000D0290020F02300208107000080240020A3
:202F400070B500255248007880210840802871D050480068504988426CD14E484030007924
:202F6000082867D34B4840300079082822D04948403000790C281DD04648403000791028FF
:202F800018D0444840300079142813D041484030007918280ED03F4840300079202809D094
:202FA0003C4840300079302804D03A484030007940286CD1374800790407240F240235488F
:202FC0008088000A0443334840300079401EA0425DD801202E4948702E4840300079801E72
:202FE00048802C48403000798873084684800120088100208872C872264A40321279511E85
:20300000234A9288501CFEF7A1F8002913D02048818820484030007908181D49C8801D4A2C
:2030200040321279511E1A4AD088FEF78FF81849C8800BE02BE0174A40321279511E144A22
:203040009288501CFEF782F81149C880114800681249086008468480002507E00D48801D05
:20306000415D0E48801D4155681CC5B2094840300079801EA842F1D8042000F065F9102001
:2030800003490870054A91881068FFF791FD70BDD0290020F0230020810700008024002043
:2030A00010B547480078A02807D045480078912803D043480078A1280ED1424800684249EC
:2030C00088420AD0414908680921FFF769FD00F077F900203A49087071E03A484030007995
:2030E00003280AD2394908680921FFF759FD00F067F900203249087061E0324800790007C3
:20310000000F002804D001282DD002284BD136E02B484078002800D050E02A48407900287C
:2031200003D101202649487003E026484079244988722348007891280BD022488079002800
:2031400004D0204880791E49087302E001201C49087391201A49087000F032F91849087BEA
:2031600000F0D2F82AE016484078002800D025E0A12013490870032000F0E6F81EE010489C
:203180004078002800D019E00D480078A02809D10E4908680821FFF703FD00F011F9002017
:2031A000074908700AE0094908680521FFF7F8FC00F006F900200249087000BF00BF10BD6E
:2031C000D0290020F0230020810700006829002070B50024484800788021084080284FD069
:2031E0004648056844480078002802D04448854246D1424940310879FFF741FA0546002D46
:2032000008D0012D04D13D4800790407240F01E03A484479394840300079A0426BDD012DB5
:203220002FD1364800790007000F002863D0334840300079401EA0425DD3304800683149F8
:2032400008602E4800790007000F8880002407E02A48401D015D2B48801D0155601CC4B269
:2032600028488088A042F3DC00202349087000F0A7F824498A8800230868891DFFF7A0FC48
:2032800039E0022D37D11D4800790007000F002831D1082C2FDB194840300179A01C8142B8
:2032A00029D31649403108792146FFF7B8F9002821D01248006813490860104840798880FB
:2032C000012408E00D48401D025D601E0D49891D0A54601CC4B20B488088A042F2DA0020DD
:2032E0000549087000F06CF806498A8800230868891DFFF765FC70BDD0290020F02300204A
:2033000081070000802400207F2807D8411CC8B27D21C90041430B4A91600EE0F12808D3F1
:20332000F92806D80107090F64225143054A916003E07D218902034A91600221014A517398
:2033400070470000E029002000B5030004F092FE0729050B11171D2329000121144A11737C
:203360001449516022E00221114A1173114951601CE003210E4A11730F49516016E0042110
:203380000B4A11730D49516010E00521084A1173002151600AE00621054A117306495160AB
:2033A00004E00021024A1173516000BF00BF00BDE029002070110100F0490200282300001B
:2033C0000020014908737047E0290020024909880918014A11807047E02900207CB500241A
:2033E0004A480078102849D149488088494988420AD94948007900090001801C46490871E1
:2034000022204249087008E043480079000900014149087120203D49087040483E490860B9
:2034200008460079F021884330303B490871084640793649897A0846374948710846807935
:203440000020887103213448403001714038056840300679002406E02F48001D005D694653
:203460000855601CC4B2082CF6D30220FFF76CFF6A4631462846FFF74FFB46E0234800789F
:20348000112842D12148807A00283ED11F48407800283AD11D4988721F48007900090001AA
:2034A0001D4908712020194908701C481A49086008460079F02188433030174908710846BA
:2034C00040791249897A0846134948710846807900208871032110484030017140380568CF
:2034E00040300679002406E00B48001D005D69460855601CC4B2082CF6D30220FFF724FFD0
:203500006A4631462846FFF707FB7CBDD029002080240020E2040000382400208907000016
:20352000244A118852888A4242D0224A52888A4204DA204A52888A1A90B207E01D4A52888A
:203540000023DB439A1A521C521890B2194A5180127B002A10D0174A5268002A0CD0154A11
:203560005268824205D9134A5268121A114B5A6002E000220F4B5A600E4A527B022A17D145
:203580000C4A9268002A0CD00A4A9268824205D9084A9268121A074B9A6002E00022054BCD
:2035A0009A60044A9268002A02D10122014B5A7370470000E029002070B505460E462C467A
:2035C0000DE072B6204604F036FFE004C00C002801D102F0F1F862B6FF34FF340234B44218
:2035E000EFD3002070BD000010B5002005490870401E054908600549086058210448FDF78E
:20360000E8FD10BD890200208C02002090020020381B0020F8B500230025009500240022AA
:2036200000BF95E001259D40ACB20D8825400095009DA54270D11A468D79012D0DD1464D9C
:2036400003263602AD192D5C012696403543424E03273F02F61935540CE03F4D03263602D9
:20366000AD192D5C01269640B5433B4E03273F02F6193554CD78002D4FD1374D60352D5C46
:20368000CE78002E01D1012600E000269640B543314E603635548D78002D2ED12E4D192660
:2036A0007601AD192D5C8E78002E01D1012600E000269640B543284E19277F01F619355475
:2036C0000D79002D0ED1244D50352D5C0E79002E01D1012600E000269640B5431E4E503665
:2036E000355424E01C4D50352D5C0E799640F6B23543194E5036355419E0174D19267601C0
:20370000AD192D5C8E789640F6B23543124E19277F01F61935540AE018E00F4D60352D5C4A
:20372000CE789640F6B235430B4E603635544D79012D0AD1084D30352D5C01269640F6B21E
:203740003543054E3036355400E000BF5D1CABB2082B00DA66E7F8BD00000440FFB581B002
:20376000074615461E4600243846029900F01CF8002802D0012005B0F0BD00240CE00A2045
:2037800060430849085CB04204D12946204600F047F803E0601C84B2232CF0D300BF002080
:2037A000E9E700002C8600000246002A03D1402901DD01207047032A03D1022901DD0120F7
:2037C000F8E7042A03D1202901DD0120F2E7052A03D1202901DD0120ECE70C2A03D1102986
:2037E00001DD0120E6E70D2A05D1012903DD402901DA0120DEE70E2A03D1202901D1012074
:20380000D8E70020D6E70000014A11547047000090000440014A11547047000080000440A6
:2038200070B5024600205EE10A235343B04C1B195B1C440004191B579B1C002B3DD00A2363
:203840005343AB4C1B195B1C440004191B195B78082B33D10A235343A54C1B195B1C4400EE
:2038600004191B5DA34CA44D6419E35C5C0864000A2353439E4D5B195B1C450045195B5D5B
:203880009C4D9D4EAD19EC540A235343984C1B195B1C440004191B5D964C35466419E35C0A
:2038A0000224A3430A245443914D6419641C45004519645D8F4DAD192B5562E00A235343D1
:2038C0008B4C1B195B1C440004191B195B78092B33D10A235343864C1B195B1C4400041925
:2038E0001B5D844C844D6419E35C4024A3430A2454437F4D6419641C45004519645D7D4DED
:203900007D4EAD192B550A235343794C1B195B1C440004191B5D774C35466419E35C8024EC
:20392000A3430A245443724D6419641C45004519645D704DAD192B5523E00A2353436C4C3B
:203940001B195B1C440004191B5D6A4C6A4D6419E35C0A245443664D6419641C45004519A2
:20396000641965780124AC40A3430A245443604D6419641C45004519645D5E4D5E4EAD1906
:203980002B550A2353435A4C1B195B1C440004191B199B788B427DD10A235343544C1B1939
:2039A0005B1C440004191B195B78082B33D10A2353434F4C1B195B1C440004191B5D4D4C76
:2039C0004D4D6419E35C012423430A245443484D6419641C45004519645D464D464EAD195E
:2039E0002B550A235343424C1B195B1C440004191B5D404C35466419E35C022423430A24F5
:203A000054433B4D6419641C45004519645D394DAD192B5564E00A235343354C1B195B1C27
:203A2000440004191B195B78092B34D10A2353432F4C1B195B1C440004191B5D2D4C2E4D2F
:203A40006419E35C402423430A245443284D6419641C45004519645D264D274EAD192B5517
:203A60000A235343224C1B195B1C440004191B5D204C35466419E35C8024A3430A2454439F
:203A80001B4D6419641C45004519645D194DAD192B5525E025E00A235343154C1B195B1CD8
:203AA000440004191B5D134C134D6419E35C0A2454430F4D6419641C450045196419657897
:203AC0000124AC402343DCB20A235343084D5B195B1C450045195B5D064D074EAD19EC54D5
:203AE00004E0431CD8B2032800D29DE600BF70BD2C86000000000440750800000149086068
:203B000070470000A802002002480068401C014908607047A4020020F3B581B006460020A2
:203B20000E49086000F01EF8044600F01BF805462F1B3046029900F0AAFF00900AE000F0CA
:203B400011F805462F1B06480068002802D004480068804700988742F1D3FEBDA4020020F6
:203B6000A80200200148006870470000A4020020034A12680260034A12680A60704700003C
:203B800050000020540000200246012000031060024800680860024870470000000000202A
:203BA000EC0200200348044A01681160001D016851607047001050009402002010B5044671
:203BC000032C00D110BD002C01D0012C7DD18121002001F0A7FB0021012001F0A3FB002159
:203BE000022001F09FFB0021032001F09BFB0021042001F097FB8021052001F093FB80219F
:203C0000062001F08FFB8021480001F08BFB0021FF20023001F086FB8121480001F082FB67
:203C20008021FF20043001F07DFB0021FF20053001F078FB0021FF20063001F073FB002158
:203C4000FF20073001F06EFB0021FF20083001F069FB00210120400201F064FB0021F348B7
:203C600001F060FB0021F148401C01F05BFB0021EE48801C01F056FB00218120800001F093
:203C800051FB0021E948001D01F04CFB0021E748401D01F047FB0021E448801D01F042FB39
:203CA00000210320000201F03DFB0021E04801F039FB8021C80001F035FB0021DD4801F066
:203CC00031FB0021DB48401C00E097E001F02AFB8021D848801C01F025FB002105200002F5
:203CE00001F020FB8121D44801F01CFB8021D248401C01F017FB0021CF48801C01F012FB06
:203D00000021CD48C01C01F00DFB0021CA48001D01F008FB80210320400201F003FB8021BE
:203D2000C64801F0FFFA8021C448401C01F0FAFA8021C248801C01F0F5FA802107200002AC
:203D400001F0F0FA0021BE4801F0ECFA0021BC48401C01F0E7FA8021B948801C01F0E2FA2C
:203D60008021B748C01C01F0DDFA8021B448001D01F0D8FA0021B248401D01F0D3FA8021AB
:203D8000AF48801D01F0CEFA81210320800201F0C9FA8021AB4801F0C5FA8021A948401CA9
:203DA00001F0C0FA8021A748801C01F0BBFA8021A448C01C01F0B6FA80210D20000201F0BB
:203DC000B1FA0021A04801F0ADFA80219E48401C01F0A8FA80210720400201F0A3FA002168
:203DE0009948FB3001F09EFA0021984801F09AFA80219648401C01F095FA14E18021002097
:203E000001F090FA0021012001F08CFA8021022001F088FA8021032001F084FA8021042040
:203E200001F080FA8021052001F07CFA8021062001F078FA8021480001F074FA0021FF2038
:203E4000023001F06FFA8021FF20033001F06AFA8021FF20043001F065FA0021FF200530D5
:203E600001F060FA0021FF20063001F05BFA0021FF20073001F056FA0021FF20083001F01A
:203E800051FA81210120400201F04CFA8021674801F048FA00216548401C01F043FA00219F
:203EA0006248801C01F03EFA00218120800001F039FA00215D48001D01F034FA00215B4867
:203EC000401D01F02FFA00215848801D01F02AFA00210320000201F025FA8021544801F074
:203EE00021FA8021C80001F01DFA0021514801F019FA00214F48401C01F014FA80214D482F
:203F0000801C01F00FFA80210520000201F00AFA8021494801F006FA80214748401C01F0AE
:203F200001FA00214448801C01F0FCF900214248C01C01F0F7F900213F48001D01F0F2F94E
:203F400081210320400201F0EDF981213B4801F0E9F981213948401C01F0E4F9812137481D
:203F6000801C01F0DFF980210720000201F0DAF98021334801F0D6F980213148401C01F00B
:203F8000D1F980212E48801C01F0CCF980212C48C01C01F0C7F980212948001D01F0C2F971
:203FA00080212748401D01F0BDF980212448801D01F0B8F980210320800201F0B3F980211D
:203FC000204801F0AFF980211E48401C01F0AAF980211C48801C01F0A5F980211948C01CDB
:203FE00001F0A0F980210D20000201F09BF90021154801F097F980211348401C01F092F90F
:2040000080210720400201F08DF900210F48401F01F088F900210D4801F084F980210B48FE
:20402000401C01F07FF900BFCCE50000010200000103000001040000010500000106000032
:2040400001070000010C0000060D0000060E000010B514480078002808D013480078FF2891
:2040600004D01248FDF7CDF80446A0470D484078002809D00C484078FF2805D00B48A030EF
:20408000FDF7BFF80446A04706488078002808D005488078FF2804D00548FDF7B2F8044689
:2040A000A04710BD006000400061004079000020B901002010B50E480079002808D00D48AF
:2040C0000079FF2804D00C48FDF79BF80446A04707484079002809D006484079FF2805D054
:2040E0000548A030FDF78DF80446A04710BD000000600040006100407E00002010B50E4832
:20410000007A002808D00D48007AFF2804D00C48FDF777F80446A0470748407A002809D069
:204120000648407AFF2805D00548A030FDF769F80446A04710BD00000060004000610040CA
:204140008300002010B50E48007B002808D00D48007BFF2804D00C48FDF753F80446A04797
:204160000748407B002809D00648407BFF2805D00548A030FDF745F80446A04710BD0000E3
:2041800000600040006100408800002010B50E48007C002808D00D48007CFF2804D00C487F
:2041A000FDF72FF80446A0470748407C002809D00648407CFF2805D00548A030FDF721F877
:2041C0000446A04710BD000000600040006100408D00002010B50E48007D002808D00D4806
:2041E000007DFF2804D00C48FDF70BF80446A0470748407D002809D00648407DFF2805D0B7
:204200000548A030FCF7FDFF0446A04710BD000000600040006100409200002010B50E4886
:20422000007E002808D00D48007EFF2804D00C48FCF7E7FF0446A0470748407E002809D0C6
:204240000648407EFF2805D00548A030FCF7D9FF0446A04710BD000000600040006100402F
:204260009700002010B50E48007F002808D00D48007FFF2804D00C48FCF7C3FF0446A047E4
:204280000748407F002809D00648407FFF2805D00548A030FCF7B5FF0446A04710BD000044
:2042A00000600040006100409C00002010B50E480078002808D00D480078FF2804D00C4852
:2042C000FCF79FFF0446A04707484078002809D006484078FF2805D00548A030FCF791FF72
:2042E0000446A04710BD00002060004020610040A100002010B50F480079002808D00E4893
:204300000079FF2804D00D48FCF77BFF0446A0470848001D407800280AD00748001D4078EB
:20432000FF2805D00548A030FCF76BFF0446A04710BD00002060004020610040A6000020C2
:2043400010B50E48007A002808D00D48007AFF2804D00C48FCF755FF0446A04707480830AB
:204360008078002809D0064808308078FF2804D00548FCF746FF0446A04710BD2060004088
:2043800020610040AB000020EB01002010B50348FCF737FF0446A04710BD0000B00000207E
:2043A00010B50F48007C002808D00E48007CFF2804D00D48FCF725FF0446A047084810306B
:2043C000407800280AD0074810304078FF2805D00548A030FCF715FF0446A04710BD0000BE
:2043E0002060004020610040B500002010B50348FCF707FF0446A04710BD0000BA00002086
:2044000010B50348FCF7FDFE0446A04710BD0000BF00002010B50F48007F002808D00E48D0
:20442000007FFF2804D00D48FCF7EBFE0446A04708481C30407800280AD007481C304078F7
:20444000FF2805D00548A030FCF7DBFE0446A04710BD00002060004020610040C400002014
:2044600010B514480078002808D013480078FF2804D01248FCF7C5FE0446A0470D48407887
:20448000002809D00C484078FF2805D00B48A030FCF7B7FE0446A04706488078002808D0D1
:2044A00005488078FF2804D00548FCF7AAFE0446A04710BD4060004040610040C90000202C
:2044C0000902002010B516480079002808D015480079FF2804D01448FCF793FE0446A04733
:2044E0000F48001D407800280AD00E48001D4078FF2805D00C48A030FCF783FE0446A0479E
:204500000748001D8078002809D00648001D8078FF2804D00548FCF774FE0446A04710BD28
:204520004060004040610040CE0000200E02002010B51648007A002808D01548007AFF2801
:2045400004D01448FCF75DFE0446A0470F480830407800280AD00E4808304078FF2805D021
:204560000C48A030FCF74DFE0446A047074808308078002809D0064808308078FF2804D0AF
:204580000548FCF73EFE0446A04710BD4060004040610040D30000201302002010B5164895
:2045A000007B002808D01548007BFF2804D01448FCF727FE0446A0470F480C304078002895
:2045C0000AD00E480C304078FF2805D00C48A030FCF717FE0446A04707480C3080780028B3
:2045E00009D006480C308078FF2804D00548FCF708FE0446A04710BD406000404061004060
:20460000D80000201802002010B51648007C002808D01548007CFF2804D01448FCF7F1FDB8
:204620000446A0470F481030407800280AD00E4810304078FF2805D00C48A030FCF7E1FDB9
:204640000446A047074810308078002809D0064810308078FF2804D00548FCF7D2FD0446C7
:20466000A04710BD4060004040610040DD0000201D02002010B50348FCF7C3FD0446A04795
:2046800010BD0000E200002010B50F48007E002808D00E48007EFF2804D00D48FCF7B1FDEC
:2046A0000446A04708481830407800280AD0074818304078FF2805D00548A030FCF7A1FD7E
:2046C0000446A04710BD00004060004040610040E700002010B50F48007F002808D00E4823
:2046E000007FFF2804D00D48FCF78BFD0446A04708481C30407800280AD007481C30407896
:20470000FF2805D00548A030FCF77BFD0446A04710BD00004060004040610040EC0000204A
:2047200010B50E480078002808D00D480078FF2804D00C48FCF765FD0446A047074840783D
:20474000002809D006484078FF2805D00548A030FCF757FD0446A04710BD000060600040F4
:2047600060610040F100002010B50F480079002808D00E480079FF2804D00D48FCF741FD42
:204780000446A0470848001D407800280AD00748001D4078FF2805D00548A030FCF731FD63
:2047A0000446A04710BD00006060004060610040F600002010B51648007A002808D01548EA
:2047C000007AFF2804D01448FCF71BFD0446A0470F480830407800280AD00E48083040783D
:2047E000FF2805D00C48A030FCF70BFD0446A047074808308078002809D00648083080786F
:20480000FF2804D00548FCF7FCFC0446A04710BD6060004060610040FB0000203B020020EE
:2048200010B50348FCF7EDFC0446A04710BD00000001002010B50348FCF7E3FC0446A0475A
:2048400010BD00000501002010B51648007D002808D01548007DFF2804D01448FCF7D1FCD4
:204860000446A0470F481430407800280AD00E4814304078FF2805D00C48A030FCF7C1FC90
:204880000446A047074814308078002809D0064814308078FF2804D00548FCF7B2FC04469E
:2048A000A04710BD60600040606100400A0100204A02002010B51648007E002808D01548AE
:2048C000007EFF2804D01448FCF79BFC0446A0470F481830407800280AD00E481830407899
:2048E000FF2805D00C48A030FCF78BFC0446A047074818308078002809D0064818308078CF
:20490000FF2804D00548FCF77CFC0446A04710BD60600040606100400F0100204F02002044
:2049200010B51648007F002808D01548007FFF2804D01448FCF765FC0446A0470F481C307A
:20494000407800280AD00E481C304078FF2805D00C48A030FCF755FC0446A04707481C3013
:204960008078002809D006481C308078FF2804D00548FCF746FC0446A04710BD6060004031
:20498000606100401401002054020020F8B505460E4600200090ECB2602C01DB0120F8BD93
:2049A000A00020181B49085C002801D00120F6E7A0002018174A8018411C3046FCF72BFCA2
:2049C0000120A1006118134A505400222846EB17DB0E1B185B115B01EB1A9B000E4FDB1934
:2049E000EF17FF0E7F197F11DA5503F051FB00222046E317DB0E1B185B115B01E31A9F000C
:204A0000064BFB18E717FF0E3F197F11DA550098C5E70000780000200060004000610040F3
:204A20000A20704703F0EAFB00281AD103208003FDF7E8FD401C002803D10C4803F004FB8D
:204A400012E0FDF783FD0A4A51681068FDF720FC002802D103F0F8FA06E0044803F0F4FA68
:204A600002E0024803F0F0FA03F05AFBA55AA55A901B002000BFFEE710B572B631218902AE
:204A8000086880F3088800BF4868804710BD70B505460E46002E05D031462846FCF756FBB0
:204AA000044600E02C46204670BD000010B50F480088002819D00D484088002815D0FFF7F2
:204AC000AFFF044601222146641C094842541C222146641C4254014608190449FCF760FB2F
:204AE0001C340121204601F0F7FA10BDFC390020F0290020F8B507460D461646FFF790FF73
:204B0000044618222146641C12484254E81CC2B22146641C0F4842543002020E2146641CC5
:204B20000C4842543004020E2146641C094842542146641C4654014608192A463946FCF7AE
:204B40002FFB601984B204480178204601F0C4FAF8BD0000F0290020C102002070B5054661
:204B60000E46FFF75DFF044619222146641C1A48425408222146641C4254310E2246641C5D
:204B800081543002020E2146641C134842543004020E2146641C104842542146641C46548C
:204BA000290E2246641C81542802020E2146641C094842542804020E2046611C8CB206494D
:204BC0000A542046611C8CB203490D5403480178204601F081FA70BDF0290020C1020020CA
:204BE000FFB587B005460E461F46002479E33019791E0840285C022809D1601C301808408A
:204C0000285C069000F028FEFFF750FF65E33019791E0840285C03287ED1601C30180840A5
:204C2000285C0690A01C30180840285CFE490870E01C3018791E0840285CFB494870201DEB
:204C40003018791E0840285CF7498870601D3018791E0840285C0007C00FF4490870601D41
:204C60003018791E0840285C4007C00FF0490870601D3018791E0840285C0011ED490870DB
:204C8000601D3018791E0840285C8007C00FEA490870601D3018791E0840285CC007C00F2D
:204CA000E6490870A01D3018791E0840285C0002E11D71187A1E1140695C0843E0490880B2
:204CC000204608303018791E0840285C00022146093171181140695C0843D94948802046AE
:204CE0000A303018791E0840285C000221460B3171181140695C0843D149888020460C307C
:204D00003018791E0840285C000221460D3171181140695C084300E016E0C949C8802046C1
:204D20000E303018791E0840285CC007C00FC549087020460E303018791E0840285C800798
:204D4000C00FC1490870C8E23019791E0840285C052819D1601C30180840285C0690BB486C
:204D600000680028EFD000200AE0A11C091889197A1E1140695CB54A12681154411CC8B2F7
:204D800006998842F1DBA8E23019791E0840285C152820D1601C30180840285C0690A01C98
:204DA00030180840285CAA490870E01C3018791E0840285CA6494870201D3018791E0840C2
:204DC000285CA3498870601D3018791E0840285C9F49C87081E23019791E0840285CC82824
:204DE00014D1601C30180840285C0690E01C30180840285C974909788842A4D1201D301873
:204E0000791E0840285C9349487066E23019791E0840285C182854D1601C30180840285CB2
:204E20000690A01C30180840285C0590059800020590E01C30180840285C059908430590B5
:204E4000059800020590201D3018791E0840285C059908430590059800020590601D3018BF
:204E6000791E0840285C059908430590A01D3018791E0840285C0490049800020490E01D26
:204E800030180840285C0499084304907248006800289FD07148006800289BD00498002851
:204EA00098D00499059840186C490968884291D869490A68059950180A460499FFF71AFE7A
:204EC0000BE23019791E0840285C19280BD1601C30180840285C06906048016860480068D5
:204EE000FFF73CFEF9E13019791E0840285C1B280BD1601C30180840285C0690E01C301873
:204F00000840285C57490870E7E13019791E0840285C1D287ED1601C30180840285C000213
:204F2000A11C71187A1E1140695C08430690E01C3018791E0840285C01284AD102A903A85B
:204F4000FEF716FE0398002842D00698401F029988423DD800200AE021460831091889198F
:204F60007A1E1140695C039A1154411C88B20699491F8142F0DC201D3018791E0840285C6C
:204F80000390039800020390601D30180840285C039908430390039800020390A01D30180E
:204FA000791E0840285C039908430390039800020390E01D3018791E0840285C0399084355
:204FC00003900698421F00231846039900F070FE10E1E01C3018791E0840285C02287DD1B4
:204FE000201D30180840285C0390039800020390601D30180840285C0399084303900398F7
:2050000000020390A01D3018791E0840285C0399084300E0F3E00390039800020390E01D39
:205020003018791E08401FE0D4020020C1020020C3020020C2020020C4020020C5020020DB
:20504000D8020020C6020020C7020020BC020020B8020020F0390020C8020020CC020020AC
:20506000D0020020C0020020285C039908430390204608303018791E0840285C02900298E9
:20508000000202902046093030180840285C02990843029002980002029020460A3030183B
:2050A000791E0840285C02990843029002980002029020460B303018791E0840285C029900
:2050C0000843029020460C303018791E0840285C0190019800020190204600E025E00D3061
:2050E00030180840285C01990843019001980002019020460E303018791E0840285C019911
:205100000843019001980002019020460F303018791E0840285C0199084301900120019B04
:20512000029A039900F0C4FD64E0E01C3018791E0840285C03282BD1201D30180840285C23
:205140000390039800020390601D30180840285C039908430390039800020390A01D30184C
:20516000791E0840285C039908430390039800020390E01D3018791E0840285C0399084393
:20518000039000231A460120039900F091FD31E0E01C3018791E0840285C04282AD1201DA2
:2051A00030180840285C0190019800020190601D30180840285C019908430190019800027C
:2051C0000190A01D3018791E0840285C019908430190019800020190E01D3018791E084010
:2051E000285C019908430190002211460320019B00F05EFD0698401C80B206906DE03019DA
:20520000791E0840285C1E2866D1601C30180840285C0002A11C71187A1E1140695C0843DD
:205220000690201D3018791E0840285C0390039800020390601D30180840285C03990843B5
:205240000390039800020390A01D3018791E0840285C039908430390039800020390E01D7C
:205260003018791E0840285C039908430390204608303018791E0840285C02900298000292
:2052800002902046093030180840285C02990843029002980002029020460A303018791EA4
:2052A0000840285C02990843029002980002029020460B303018791E0840285C029908434A
:2052C000029000220220029B039900F0F1FC0698401C80B2069000E007E00698801C2018E7
:2052E00084B20998844200DA81E400BF0BB0F0BD10B501231A4600211846FCF72BFD0122A5
:2053000011461046FCF78AFDFBF7DCFE034802F0A9FF02480249086010BD00000090D00388
:20532000A0020020F0B585B005460C460020C0430390EFB22804060E0F2E45DA082F43DAED
:205340000120B8406946888080202040002816D101208871A007800F022801D1487209E07F
:20536000A007800F012802D16946487202E0002069464872F0B201A9FEF74CF922E000207F
:20538000694688710E202040002800D000BF10202040002802D16946087202E001206946BA
:2053A0000872E007C00F002802D16946887202E0012069468872304600F026F801A90090AF
:2053C000FEF728F900200390039805B0F0BD000001220B490A710A720A730A740A750A769F
:2053E0004A714A724A734A744A754A76002004E000218200034B9950401C0C28F8D370474C
:2054000000610040A813002000B501460B0002F031FE10090B0D0F111315172525191B1FBB
:2054200021231D2500201AE0012018E0022016E0032014E0042012E0052010E006200EE045
:2054400007200CE00A200AE00B2008E00F2006E00C2004E00D2002E00E2000E000BF00BF52
:2054600000BDFEB504460E460020C0430190E5B22004070E0F2F17DA082D15DA0120A8403E
:2054800085B2002E07D13846FFF7BEFF29460090FEF7BAF906E03846FFF7B6FF29460090E9
:2054A000FEF7B8F9002001900198FEBD10B505480068002802D003480068804700F03EFC29
:2054C00010BD00004400002070B504460D46601E0D49884200D90124002C00D101244020BB
:2054E0000A490870084600786043094948610321081F02F0D9FD0020054988610720086183
:205500000448056070BD0000FFFFFF004800002000E000E0440000200020C043002809DBF5
:20552000C206D20E01219140054A1160BFF34F8FBFF36F8F00BF002002490861886170479D
:2055400080E100E000E000E0F0B587B006460C46002700216846C182002003906846818233
:20556000418201824183018300F0FAF8032E7DDA206800287AD060680028FBD0002E04D07C
:20558000012E3ED0022E72D17CE0674D00231F2202210520FEF7E2F800231E220121052026
:2055A000FEF7DCF8022168468180002181710172012181720021C17101A90520FEF72AF87C
:2055C00001216846818081710021C17101A90520FEF720F8606803900721684601821021F4
:2055E0004182002181824183802101833221C1824E490A20FFF7CAF94D490B20FFF7C6F955
:2056000081E0494DAD1C0023032204211846FEF7A5F80023042208211846FEF79FF80421EC
:2056200068468180002181710172012181720021C17101A90020FDF7EDFF0821684681804B
:20564000012181710021C17101A90020FDF7E2FF606803900721684601821021418200217B
:205660008182418380210183322101E058E049E0C18230490D20FFF789F92F490E20FFF7AC
:2056800085F940E02D4D10232E2240210720FEF765F811232F2280210720FEF75FF880215B
:2056A00068468180002181710172012181720021C17101A90720FDF7ADFF402168468180CC
:2056C000012181710021C17101A90720FDF7A2FF6068039007216846018210214182002134
:2056E00081824183802101833221C1821449E068C86014490720FFF749F913490820FFF725
:2057000045F900E000BF00BF03A9284601F0FAF80746002F04D0CD220CA1384602F068FE2E
:20572000606807B0F0BD000010100000D16600007D66000079670000256700001020000067
:205740009813002021680000CD6700002E2E5C7372635C5254455F554152542E630000004E
:2057600000200F49086048600872C8600D49086048608860C8600C49086048600872C86082
:205780000A49086048608860C8600949086048600872C8600749086048608860C86070476B
:2057A00048130020781300205813002088130020681300209813002010B502F03FFC10BD58
:2057C0001A20084908722B2048723C2088724D20C8727F20044909680860AC20034948702D
:2057E0007047000000040240400000200010024070B504460025204600F007F8064630464F
:20580000FCF76CFE85B2284670BD01460868704710B504460F488088002800D110BD0D4862
:205820000088182250430B4A0832811818222046FBF7B6FC07490988481C1721FBF79CFCA0
:2058400088B20449088008468088401E88800120E4E70000F013002000200549086005494A
:2058600008600549087005490870054908707047B0020020B4020020C1020020C202002048
:20588000C402002010B519480078012813D118480078012804D100201549087015490870D5
:2058A00014480078322801DB02F03AFC11480078401C1049087010480078012814D10F4883
:2058C000007864280BD300200B4908700C480078801E0B49087000200849087004E00748A8
:2058E0000078401C0549087010BD00007402002076020020750200207A0200207B02002043
:2059000088020020F8B504460D460026002700200090201300F09AF900901448844205D059
:20592000801C844202D01248844217D122202840222806D127073F0F39460098FBF766FE77
:2059400006461220284012280ED12007000F471C39460098FBF75AFE064605E02107090FDD
:205960000098FBF753FE06463046F8BD1010000010200000FFB58BB01C46002007900690E7
:2059800005903848049010210B980840002801D0022707E040210B980840002801D00127CC
:2059A00000E00027002C04D0149804700120089001E010200890002548E0002C08D02546A2
:2059C0006000294A115A0C98FBF7C0FB079006E06800254A115A0C98FBF7B8FB07903E4615
:2059E00030E0711C0798FBF7B1FB400806900D98FBF795FC03900D9A0699881AFBF78FFCCF
:205A000018490190FBF710FC02900399FBF749FC05900598FBF78AFC4900490803910290C7
:205A20000498FBF783FC4900490801910090039B029AFBF78FFC03D20A95099605980490A2
:205A4000701CC6B27F2ECCDD681CC5B208988542B3DB14990A980870149909984870049893
:205A60000FB0F0BD0000C8428A87000010B50246374BD01A9A4233D014DC364BD01A9A4210
:205A80002DD008DC34481018002846D002284CD010285AD11DE0012827D002282BD01F2811
:205AA00053D117E02B4C423C031BA04229D009DC01281BD002281FD0274B4133C0180028E5
:205AC00043D13AE0012B22D0202B1BD0212B3CD11EE000BF214803890B43038136E000BF92
:205AE0001E4843890B43438130E000BF1B4883890B4383812AE000BF1848C3890B43C381CB
:205B000024E000BF164883880B4383801EE000BF1348C3880B43C38018E0104843890B43AA
:205B2000438103890B43038110E00C48C3890B43C38183890B43838108E00948C3880B43F1
:205B4000C38083880B43838000E000BF00BF10BD4110000021100000F0EFFFFF00110440C7
:205B60000014044030B502460020334C131BA24233D014DC314C131BA2422DD008DC304B11
:205B8000D318002B46D0022B49D0102B51D11DE0012B27D0022B2BD01F2B4AD117E0274D1E
:205BA000423D5C1BAB4229D009DC012B1BD0022B1FD0234C41341B19002B3AD134E0012C62
:205BC00022D0202C1BD0212C33D11EE000BF1D4B1C880C40E0B22DE000BF1A4B5C880C4043
:205BE000E0B227E000BF174B9C880C40E0B221E000BF144BDC880C40E0B21BE000BF124B71
:205C00001C880C40E0B215E000BF0F4B5C880C40E0B20FE00B4B5C880C40E0B20AE0094BED
:205C2000DC880C40E0B205E0074B5C880C40E0B200E000BF00BF30BD41100000211000005C
:205C4000F0EFFFFF001104400014044030B50246002100230024002000BF0BE001258D4068
:205C6000EBB215461D402C469C4201D1084603E04D1CE9B20429F1D300BF30BD00BF0948CB
:205C80000068094948430949401806490860084600680028F3D008460068401C0028EED0C5
:205CA00070470000800200206D4EC6413930000030B50F4C21600F4C22600F4C23600028BC
:205CC00003D102240D4D2C7010E0012803D103240A4D2C700AE0022803D10424074D2C70CD
:205CE00004E0032802D10524044D2C7030BD0000580000205C000020600000204C000020DF
:205D000010B504480068401E02490860FFF7CEFB10BD00007400002010B5FFF7B3FD10BDA1
:205D200010B50A20FCF7A6F910BD704710B57D200001FDF74BFB10BD7047704710B5FDF7CD
:205D4000E3FE0F480068401C0D49086008460068142806D3002008600A480068401C0949CE
:205D6000086009480088401C0749088008460088282804DB002008800220FBF7EDFB10BD38
:205D800070020020680200206C0200200CB500BF054800680090044800680190019900981D
:205DA0008842F5D100980CBD6402002010B5FBF759FCFCF77EFC00F0B7FF10BD70B53148E2
:205DC00000683149096840182E490860084600687D21C900884211D32A480068FBF7B6F9F3
:205DE00006467D21C90027480068FBF7AFF925480160264800688019244908602448406859
:205E00002149096840182249486008460068002837D10025084684682EE02068002829D040
:205E20001B49606849680022D243511A884205D21749606849684018606002E00020C0434C
:205E40006060A1686068884214D3206801280AD100202060002D03D10D492069886004E028
:205E60002069286101E000206060E068002801D0E068804725462469002CCED100200449CF
:205E8000486070BD600200205C020020640200204816002010B5FFF73FFB322000F008F8F2
:205EA00002493220FFF710FB10BD0000BD5D000010B504460D48046000200D4908600D4961
:205EC00008600D49086048608860FFF75FFF0B4908600020486088600120C8600320086177
:205EE000052048610720886110BD00005C0200206002002064020020481600202C16002091
:205F000070B5FFF753FFFFF741FF05463A480068A84203D8384800682C1A06E036480068EA
:205F20000021C943081A4019441C33480560406800193149486008464068022806D308464F
:205F40000079C007C00F4860FFF7F0FE2A48806800192949886008468068052807D38868AC
:205F60000521FBF7F3F824488160FFF7E6FE2248C06800192049C8600846C0680A2807D339
:205F8000C8680A21FBF7E2F81B48C160FFF7C8FE19480069001918490861084600691428FA
:205FA00007D308691421FBF7D1F813480161FFF7BCFE1148406900190F4948610846406926
:205FC000322807D348693221FBF7C0F80A484161FFF7B2FE0848806900190749886108466C
:205FE0008069642807D388696421FBF7AFF802488161FFF791FE70BD2C1600201FB5FFF739
:20600000DFFBFFF775F9FFF745FF0C48FDF776FDFFF7DEF90020FDF7D1FD01200090E120EC
:2060200040020190002002900548039069460220FFF78AFAFCF76AF81FBD0000B95700006F
:206040003516000010B580201B4948711A201A49203908722B2048723C2088724D20C87201
:20606000002016494860FBF709FF154908600020C04314490860144908601448144908606B
:20608000114903221202891848600F49891888600D498918C8600C49891808610A498918D1
:2060A000486109498918886107498918C861AC200849487010BD00002004024000B0014048
:2060C000A002002080E200E000E100E0C0C0C0C000E400E000100240F3B583B007463C463B
:2060E00002940498002845D00A2C3FDD0020C04322460A3A01231B030A2100901E48FBF7BB
:2061000067FF064625460024EB222146641C1A48425490222146641C42542804020E214680
:20612000641C154842542146641C45542812C043C2B22146641C10484254E843C2B22146E0
:20614000641C0D484254310E2246641C81543002020E2146641C084842543004020E21461E
:20616000641C054842542146641C46540248029901F05CFF05B0F0BDF0290020F8B5034679
:206180000C460021012000900025608922263040222826D10720014319812021A07A00076D
:2061A000000F0143084628430146198204214803014320890143A0890143E0880143A0880F
:2061C0000143198321200001C05A7F267602B043567876027F277F023E4030432126360197
:2061E000F05260891226304012283BD100210720014359813F48007C012630433D4E307454
:20620000202108462843014600BFB0150143E08901430220014300BF59820421400301431C
:2062200020890143A089014310200143A088014359833148C05A7F267602B043567876025F
:206240007F277F023E4030432B4EF052998EE089002804D10E4600988643314601E0009839
:2062600001439986608912263040122804D1988C80088000801C988460892226304022284C
:2062800004D1988C80088000401C9884DE8C0020DE8C360936010643DE84D88C0009000102
:2062A00016783607360F3043D88460891226304012280BD1588D0226B0435885188DB043E3
:2062C0001885588C80088000801C588460892226304022280BD1188D012630431885588D35
:2062E00030435885588C80088000401C58840020F8BD00006004044012020000F8B50346A3
:206300000C460021042000904503608922263040222826D10720014399812021A07A000745
:20632000000F0143084628430146998204214803014320890143A0890143E0880143A0880D
:206340000143998385208000C05A7F267602B043567876027F277F023E4030438526B600CF
:20636000F05260891226304012283BD1002107200143D9815448007C04263043524E307425
:20638000202108462843014600BFB0150143E08901430220014300BFD9820421400301431B
:2063A00020890143A089014310200143A0880143D9834648C05A7F267602B0435678760249
:2063C0007F277F023E403043404EF052998EE089002804D10E4600988643314601E00098A3
:2063E00001439986608912263040122804D1988C0C26B04308309884608922263040222812
:2064000004D1988C0C26B043001D9884DE8C3606360F00263601F0273E403046DE8CBE4367
:206420000643DE84D88CF026B043167836013E403043D88460891226304012281ED15E8D8D
:206440003607B60F0227BE43B6000C273E4030465E8DBE4306435E851E8D3607B60F022745
:20646000BE43B6000C273E4030461E8DBE4306431E85588C0C26B043083058846089222658
:20648000304022281ED11E8D3607B60F01273E43B6000C273E4030461E8DBE4306431E8588
:2064A0005E8D3607B60F01273E43B6000C273E4030465E8DBE4306435E85588C0C26B04348
:2064C000001D58840020F8BD6004044016020000F8B503460C460021012000900025608906
:2064E00022263040222825D10720014399802021A07A0007000F01430846284301461981D1
:2065000004214803014320890143A0890143E0880143A08801439981F000C05A7F26760214
:20652000B043567876027F277F023E403043FF261136F05260891226304012283DD1002162
:2065400007200143D9804C48007C102630434A4E3074202108462843014600BFB015014379
:20656000E08901430220014300BF598104214003014320890143A089014310200143A088CD
:206580000143D981FF201330C05A7F267602B043567876027F277F023E403043FF26133605
:2065A000F052198CE089002804D10E4600988643314601E000980143198460891226304077
:2065C000122804D1988A80088000801C9882608922263040222804D1988A80088000401C86
:2065E0009882DE8A0020DE8A360936010643DE82D88A0009000116783607360F3043D88229
:20660000608912263040122817D15E8B0227BE43B007800F5E8BB608B60006435E831E8B3E
:20662000BE43B007800F1E8BB608B60006431E83588A80088000801C58826089222630400B
:20664000222817D11E8B01273E43B007800F1E8BB608B60006431E835E8B3E43B007800FB9
:206660005E8BB608B60006435E83588A80088000401C58820020F8BD600404401CB5002005
:206680000F49087307210F4800F028F9009069460878002807D007210A4800F017F96846B1
:2066A000007801F0A8FE0848807C01900748C068002804D00548C1686846007988471CBD36
:2066C0002060004010100000001304407813002010B500200F4908720F4800680E4949685A
:2066E00088420BD20C4801680068401C0A4A10601046C068405C0949087409E0002006496E
:20670000087207488068002802D005498868804710BD00002060004048130020001304406A
:20672000781300201CB500200F49087607210F4800F0D4F8009069460878002807D00721C6
:206740000A4800F0C3F86846007801F054FE0848807D01900748C068002804D00548C1680C
:206760006846007988471CBD2060004012100000001304408813002010B500200F4908759C
:206780000F4800680E49496888420BD20C4801680068401C0A4A10601046C068405C0949DA
:2067A000087509E000200649087207488068002802D005498868804710BD000020600040C7
:2067C0005813002000130440881300201CB500200F49087007210F4800F080F80090694635
:2067E0000878002807D06846007801F004FE0721084800F06BF80848807C01900748C068E2
:20680000002804D00548C1686846007988471CBD2060004010200000001504409813002023
:2068200010B500200F4908770F4800680E49496888420BD20C4801680068401C0A4A1060E9
:206840001046C068405C0949087409E000200649087207488068002802D005498868804748
:2068600010BD000000600040681300200015044098130020002006490988602211400029F0
:2068800003D10449097A002900D0012070470000001404406813002010B503460C46FFF73A
:2068A000E9FF00280CD101200649086008464460012008720846C360C068007802490874AE
:2068C00010BD0000681300200015044070B504460D4629462046FFF7C9F870BD70B505460C
:2068E0000E4631462846FFF73DF9002801D0012400E00024204670BD014800687047000016
:20690000A0020020F0B585B004460D460020039069892046FEF7F6FF40B203900398002801
:2069200002D0039805B0F0BD55482018002809D002282DD001210903401A4FD04900401A41
:2069400072D172E0A0120121FBF748FA4D4FFFF7D3FF019002A80090F88C03071B0F2A6821
:2069600020460199FFF706F806463046FAF7DEFC0022454B01910090FAF7ECFC02D20520F0
:20698000C043CFE702AA29463846FFF7F7FB73E0A0120121FBF722FA3A4FFFF7ADFF0190CC
:2069A00002A80090F88C0006030F2A6820460199FEF7E0FF06463046FAF7B8FC0022324B95
:2069C00001910090FAF7C6FC02D20520C043A9E702AA29463846FFF791FC4DE0A012012139
:2069E000FBF7FCF9294FFFF787FF019002A80090F88A03071B0F2A6820460199FEF7BAFFFB
:206A000006463046FAF792FC00221F4B01910090FAF7A0FC02D20520C04383E702AA294679
:206A20003846FFF755FD27E025E0E0120121FBF7E5F9174FFFF760FF019002A80090F88A98
:206A400003071B0F2A6820460199FEF793FF06463046FAF76BFC00220B4B01910090FAF744
:206A600079FC02D20520C0435CE702AA29463846FFF72EFD00E000BF00BF039852E7000076
:206A8000F0EFFFFF001104400000F03F00140440001604401FB504460A4800900021684614
:206AA000417108218171032101727F21417284727821C172AA21017341738173C173FBF750
:206AC000B7FB1FBD8907000000B503460A46002A03D1184600F000F903E00121184600F0B2
:206AE000FBF800BD7047F0B505460E4617461C46002C05D13A463146284600F0EFF805E009
:206B000001233A463146284600F0E8F8F0BD70B504460D461646324629462046FCF75CF8BD
:206B200070BD000010B50020044908700449087004490860FCF758FD10BD00007C02002051
:206B40007D020020840200201CB5002001904848007A00287ED000204649087046480079C0
:206B600031282DD008DC10280FD011284CD0222814D027285AD11AE034282AD0362831D018
:206B8000372838D03E2851D147E0394A203AD18C394A1068521D00F0CBF859E0344A203A77
:206BA000D18C354A1068521D00F00CFA50E0304A203AD18C304A1068521D00F0F9FA47E050
:206BC0002B4A203AD18C2C4A1068521D00F024FC3EE0274A203AD18C274A1068521D00F08E
:206BE0007FFE35E0224A203AD18C234A1068521D00F084FF2CE01E4A203AD18C1E4A10680E
:206C0000521D01F0AFF823E0194A203AD18C1A4A1068521D00F044F91AE0154A203AD18CC8
:206C2000154A1068521D01F0FBF811E012480068124988420BD01120019001A80E49009025
:206C4000087901230D4A563A194601F067F900BF00BF00E00BE000200549087208480078FF
:206C6000012804DD012007490870024908701CBD8820002074020020A81B0020DF0700005E
:206C800077020020760200201FB51048007801281BD10F4800900021684641710821817187
:206CA0000621017250214172022181720021C1723221017301214173F4218173AA21C17307
:206CC000FBF7B6FA0120034908701FBD79020020890700007402002070470000F0B50446EA
:206CE000002B12D10125094E3572094D2C60551E203EF584002006E00E78054D2D1D2E548C
:206D0000491C451CA8B29042F6DBF0BD88200020A81B002070B504460D4616463246294653
:206D20002046FFF7F4FE70BD10B5FFF70DFF10BDF7B584B00E461020039000243746049810
:206D4000029000200190002F03D113204F49087002E000204D4908704C48007800281AD17B
:206D6000002505E00698405D49494855681CC5B2BD42F7DB4648007880210840C00901908A
:206D8000434800784406640E002C01D0032C02D912203E4908703D480078002804D1012FD2
:206DA00002D013203949087038480078002812D1022C07D13748007801280CD17E203349B4
:206DC000087008E0032C06D132480078022802D17E202E4908702D48007800282AD12C494C
:206DE0004870322088700120C870F4200871012C10D10198002807D108460523264A0021FD
:206E00000090039801F08AF832212448FCF784FE01F086F9FFF786FE1E480470019800281B
:206E200032D11B4805231C4A00210090039801F075F829E018495631029888421CD1134817
:206E40000078112820D01148007812281CD00F4800787E2818D00D4800787F2814D00B4892
:206E60000078312810D0094801230B4A19460090039801F053F807E004480123064A1946CB
:206E80000090039801F04AF807B0F0BD7802002054160020770200208907000050C30000D0
:206EA000F7B586B006460F4611200590002004903D46039602903E480078012803D17F208D
:206EC0003C49087002E000203A49087039480078002804D1012D02DA132036490870354811
:206EE000007800281AD1002405E00898005D32490855601CC4B2AC42F7DB2F4800788021E7
:206F00000840C00902902C4800784006400E04900498012802D01220264908702548007825
:206F2000002804D1012D02D013202249087021480078002810D10298002837D11E48012300
:206F40001E4A00210090059800F0E8FF32211C48FCF7E2FD01F0E4F8184956310398884201
:206F60001CD114480078112820D01248007812281CD0104800787E2818D00E4800787F285C
:206F800014D00C480078312810D00A4801230B4A19460090059800F0C1FF07E005480123A9
:206FA000064A19460090059800F0B8FF09B0F0BD770200207802002054160020890700009B
:206FC00050C30000F7B584B00E4622200390374604980290022F03DA13206949087002E09D
:206FE00000206749087066480078002822D1002505E00698405D63494855681CC5B2BD4280
:20700000F7DB6048007804025E4949780C435E4884420FD05C480E3084420BD0801E84428F
:2070200008D0801D844205D05848844202D031205349087052480078002804D1022F02D091
:2070400013204F4908704E48007800286BD14E490C31601A8C422CD008DC4D48201800288A
:2070600045D04C494018002850D104E0022811D006284BD12CE00F2247494248801CFAF7A8
:207080008FF840481123454A00210090039800F045FF47E0092242493A48801CFAF780F83A
:2070A00038480B233D4A00210090039800F036FF38E009223B493348801CFAF771F8314879
:2070C0000B23364A00210090039800F027FF29E0042235492B48801CFAF762F829480623FF
:2070E0002E4A00210090039800F018FF1AE00D222E492448801CFAF753F822480F23274AD4
:2071000000210090039800F009FF0BE031201C49087008460123214A19460090039800F0BB
:20712000FDFE00BF29E01D495631029888421CD113480078112820D01148007812281CD05B
:207140000F4800787E2818D00D4800787F2814D00B480078312810D0094801230F4A194649
:207160000090039800F0DAFE07E0054801230B4A19460090039800F0D1FE07B0F0BD0000C2
:20718000780200205416002087F1000024100000DCEFFFFF9D1EFFFF3C8C00008907000045
:2071A0004B8C0000548C00005D8C0000618C0000F7B586B00746272003900024079E0297D7
:2071C0008B48029F874203D111208A49087002E000208849087087480078002806D18648C3
:2071E0000078022802D07F208249087081480078002804D1002E02D113207E4908707D48C3
:207200000078002812D1002505E00898405D7B494855681C85B2B542F7DB78480478112C46
:2072200004D0122C02D01220724908707148007800280CD1112C05D1012E08D013206D49CC
:20724000087004E0052E02D013206A49087069480078002808D1122C06D1694800780128DE
:2072600002D024206349087062480078002808D1112C06D163480078012802D137205D4981
:2072800008705C48007800287ED1112C02D0122C7BD142E05C480078022808D11120574938
:2072A0000870002048708870C870087116E0FEF7E5FC56480068000E5049487053480068A1
:2072C0000002000E8870514800880004000EC8704E480078087101204949087047480523D2
:2072E000434A563A00210090039800F017FE434841786846017441488178684641743F484D
:20730000C178684681743D4801796846C17404A8FAF782FE3E49086059E000203849087051
:2073200036484078000635498978090408433349C9780902084331490979084305903449CE
:207340000598096888420CD102202F4908702B480123274A563A00210090039800F0DEFDB7
:2073600027E02C480078401C2A49087008460078032812DB01202349087036201D490870BC
:20738000084601231A4A01E022E013E0563A19460090039800F0C2FD0BE035201549087062
:2073A00008460123124A563A19460090039800F0B5FD0CE012200F490870084601230C4A8D
:2073C000563A19460090039800F0A8FD00BF0DE007495E390298884208D106480123044A6E
:2073E000563A19460090039800F098FD09B0F0BDDF070000780200207702002054160020E5
:207400007C0200207A0200207D020020800200208402002088020020F7B58AB031200390D7
:20742000002002900B9D0A9801900026F7490198884203D11120F649087002E00020F449FB
:207440000870F3480078002806D1F2480078022802D07F20EE490870ED480078002806D15A
:20746000ED480078022802D03320E9490870E8480078002804D1032D02D21320E4490870E5
:20748000E3480078002812D1002405E00C98005DE2490855601C84B2AC42F7DBDF4800789B
:2074A00002900298012802D01220D9490870D848007800283FD1D94840780002D74989780D
:2074C00008430646FF20000286422BD1D34800790006D249497909040843D049897909023B
:2074E0000843CE49C97908430990CC48007A0006CA49497A09040843C849897A09020843D8
:20750000C649C97A08430890032189030998884204D11D218903089888420CD93120BC49D7
:20752000087008E0BE48864205D0BE48864202D03120B7490870B6480078002822D1F01F3F
:20754000FF38FC3800280CD0B7494018002802D0012812D10BE00C2D02D01320AC490870C8
:207560000FE0072D02D01320A949087009E0032D02D01320A649087003E03120A44908705B
:2075800000BF00BFA248007800287DD1F01FFF38FC38002806D0A4494018002875D0012842
:2075A00074D14FE19D48C07800069C490979090408439A494979090208439849897908434B
:2075C00005909A48007D002840D199480068C0439749086005980968884227D195480078C5
:2075E0003E2813D10020C0439149086001218F48017500208949C87008460423834A563A71
:2076000000210090039800F089FC65E000218748017501208149C870084604237B4A563A11
:2076200000210090039800F079FC55E000217F48017501207949C87008460423734A563A29
:2076400000210090039800F069FC45E077484038008A76494039498A884208DB73484038B8
:20766000008A72494039498A401A80B206900698002807D06D4940394A8A1431501806996B
:2076800000F06CFD6A4802E012E126E003E10068C043674908600598096888420CD10020C8
:2076A0005E49C87008460423584A563A00210090039800F033FC0BE001205849C8700846A6
:2076C0000423524A563A00210090039800F026FC0020C04356490860E9E05448007D0128C4
:2076E00073D10398FFF7D6F9FAF75EFFFAF72EFF00200790504880680121C904884205D2B3
:207700004D48006861214902884212D04B48806823214903884205D2484800686121490282
:20772000884202D0012007901FE0FAF7E9FE07901BE0414A51681068FAF7AAFD002811D12E
:2077400003208003FEF754F8074623204003FEF74FF8874202D10120079006E0FAF7D0FE3A
:20776000079002E0FAF7CCFE0790079801282DD1334800F069FC2321490303208003FBF780
:207780001BFF0490049800280FD101212748417500202249C870084604231C4A563A002101
:2077A0000090039800F0BAFB2FE000211F48417501201A49C87008460423144A563A00216C
:2077C0000090039800F0AAFB1FE00FE000211748417572200E490870084601230B4A563A0D
:2077E00019460090039800F099FB0EE000210F48417501200949C87008460423034A563A62
:2078000000210090039800F089FB50E0DF07000078020020770200207D0200205416002036
:207820000202000001FF00000203FFFF781B00208C020020890200209C1B0020901B002093
:20784000A55AA55A224A91685068FAF721FD002811D10398FFF71EF9002000F0F5FB00202C
:207860001C49C870084604231B4A00210090039800F054FB0EE00021154840300175012093
:207880001449C87008460423134A00210090039800F044FB0BE03120104908700846012387
:2078A0000D4A19460090039800F038FB00BF0CE0094908390198884207D108480123064A87
:2078C00019460090039800F029FB0DB0F0BD0000381B002054160020890700007802002079
:2078E000F7B586B006460025002734200590079804900396784802907848039E864203D10A
:2079000011207749087002E000207549087074480078002806D173480078022802D07F20C5
:207920006F4908706E480078002806D16E480078022802D033206A490870694800780028F1
:2079400005D104980A2802D013206549087064480078002815D1002405E00898005D634974
:207960000855601C84B204988442F6DB5F480078002803D15D484078442802D0312058491D
:2079800008705748007800287ED1594908705748807800065549C9780904084353490979D5
:2079A0000902084351494979084305464F48807900064E49C979090408434C49097A090295
:2079C00008434A49497A084307464A48007D01284AD14848407D012839D10320800385422E
:2079E00028D11D208003874224D2424840380560E81DFF30FA303F4940394860F81FFF3853
:207A0000FA388860202039490870042048700220887008460323314A563A0021009005984F
:207A200000F07CFA012133488175002031494039C8604FE031202A49087008460123274AC4
:207A4000563A19460090059800F068FA42E070202349087008460123204A563A19460090C7
:207A6000059800F05BFA35E02348854217D1202F15D101211F48817520201C490870042000
:207A800048700220887000E016E008460323134A563A00210090059800F040FA1AE031201A
:207AA0000F490870084601230C4A563A19460090059800F033FA0DE008495E3903988842BB
:207AC00008D107480123054A563A19460090059800F024FA09B0F0BD02040000DF0700008F
:207AE00078020020770200207D0200205416002089020020781B002000009F01F7B596B03A
:207B0000064600201590149036200390179D02968C48029E864203D111208B49087002E00C
:207B200000208949087088480078002806D187480078022802D07F2083490870824800782C
:207B4000002806D182480078022802D033207E4908707D48007800280FD1681E7D49C8609D
:207B60000846C068002805D00846C06801218902884202D913207449087073480078002807
:207B800020D1002405E01898005D73490855601C84B2AC42F7DB704801786E484030807DFF
:207BA00081420CD16B484030807D159069484030807D401CC1B267484030817502E07320E9
:207BC000614908706048007800287DD161484030007D012879D15F4800680321890388425B
:207BE00054D35C4800680121C90488424ED2002447E01898001941785648028A1430815469
:207C00001438008A401C53490882084600685349884234D24F48008A402830D3FF224021DC
:207C200004A8F9F7CFFA00270CE04A48418A1430405C04A9C8554748408A401C45494882B8
:207C4000781C87B2402FF0D340214248143000F085FA72B63F4904AA0868402100F02EFC3E
:207C6000149062B61498002808D13A48006840303849086000200882488200E005E0601CA3
:207C800084B23448C068A042B3D80DE072202E490870084601232B4A563A1946009003982E
:207CA00000F03CF919B0F0BD149800280ED12A491598087008460123224A563A00210090BF
:207CC000039800F02BF93BE02CE00CE072201E490870084601231B4A563A19460090039880
:207CE00000F01CF9DEE7012408E01B48005D1C49097840181A490870601C84B2AC42F4DB65
:207D0000691E1548401C00F029FA134915980870084601230B4A563A00210090039800F0FC
:207D2000FDF80DE007495E390298884208D106480123044A563A19460090039800F0EEF88D
:207D400000BFAFE7DF07000078020020770200207D020020381B002054160020C0FF070053
:207D600089020020FEB504460D46372001902F4626462548864203D111202449087002E03E
:207D800000202249087021480078002806D120480078022802D07F201C4908701B480078CD
:207DA000002806D11B480078022802D033201749087016480078002804D1002F02D01320BB
:207DC000124908701148007800280ED1FAF7E0FA002111488175114800230B4A563A1946FD
:207DE0000090019800F09AF80CE007485E38864208D106480123044A563A1946009001988E
:207E000000F08CF8FEBD0000DF07000078020020770200207D020020781B0020541600203E
:207E2000F7B586B007460D463E200590002004902E4603970290002E03D11320344908704F
:207E400002E00020324908703148007800281AD1002405E00898005D2E490855601CC4B25D
:207E6000B442F7DB2B48007880210840C0090290284800784006400E04900498002802D065
:207E800012202349087022480078002804D1012E02D013201E4908701D48007800280BD1F9
:207EA0000298002832D11B4801231B4A00210090059800F033F829E0174956310398884253
:207EC0001CD113480078112820D01148007812281CD00F4800787E2818D00D4800787F28F1
:207EE00014D00B480078312810D0094801230A4A19460090059800F011F807E004480123F5
:207F0000054A19460090059800F008F809B0F0BD780200205416002089070000FFB581B097
:207F2000064617460A9D0298002822D0224807607F202149087108464671403104988884CC
:207F4000002406E029781C48801D01556D1C601C84B219484030808CA042F3DC1649403186
:207F6000898C891C8AB214490868091DFEF7D2FE20E012480760402030431049087140317C
:207F800004988884002406E029780C48401D01556D1C601C84B209484030808CA042F3DCCE
:207FA00006494031898C491C8AB204490868091DFEF7B0FE05B0F0BDFC2000209420002053
:207FC00010B500200D4908700D4908700D4908700D4908700D480E49086000200D49087082
:207FE0000D4908700D4908600D4908700D4908700D490870FBF7F8FA10BD00007602002042
:2080000075020020740200207802002058D93401800200207C0200207D02002084020020AE
:20802000880200207B0200207A02002070B504460D4629462046FEF72FFC70BDAC20014963
:20804000487070470010024010B5044606480749086008464460064800F0EDF9034A0821BE
:20806000034800F006FA10BDA55A7AA7940200200010500030B47446641E2578641CAB4298
:2080800004D3635D5B00E31830BC18471D46F8E7002805DBC206D20E01219140014A116007
:2080A0007047000080E200E010B5002819DB1A4A03231B02D21883089B00D2588307DC0E91
:2080C000FF23A3409A438B071B0E8407E40EA3401A43114B032424021B198408A4001A51CE
:2080E00018E00E4A03071B0F083B9B089B00D2588307DC0EFF23A3409A438B071B0E8407B5
:20810000E40EA3401A43054B0407240F083CA408A4001A5110BD000000E100E01CED00E029
:20812000BFF34F8F03480449C860BFF34F8F00BF00BFFDE70400FA0500ED00E002E008C87B
:20814000121F08C1002AFAD170477047002001E001C1121F002AFBD17047000010B5024614
:208160000EE01378521C094C247863401B069B0D074CE358054C2468240A6340034C2360AD
:208180000B46491E002BECD110BD00008C0200203C88000010B50021024841700248F9F7E5
:2081A0004BFB10BD246000400054044010B500210D48417002210D48F9F7C2FB002812D035
:2081C00002210A48F9F790FB09490848F9F70AFD0848FDF71DFB08480068002803D00548BA
:2081E00005490968884710BD5C60004000540440F0130020D81300206800002070B5002590
:2082000061246402202221461548F8F7EDFF002823D120222146403111484030F8F7E4FFC1
:2082200000281AD12022A1180D482030F8F7DCFF002812D120222146603109486030F8F7AC
:20824000D3FF002809D110222146803104488030F8F7CAFF002800D100E00125284670BDB2
:20826000AC87000010B5044603492046F8F76EFF0249087010BD000040420F005802002013
:2082800070B50446002C01D1064D01E0012070BD2846F9F72CFB032801D10220F7E700204D
:2082A000F5E700000054044072B60120000309498860BFF35F8F62B6FAF74EF8FAF7ACF840
:2082C000FDF79CFEFEF7E0FC03E0FDF775FAFDF717FEFAE700ED00E00346002B01D10B4AA7
:2082E00001E0012070475020815A094801400720014350208152815A05480140FF20013081
:208300000143502081520020ECE7000000540440F8F8000010B588B0044623231F2202216A
:208320000520FBF71BFA22231E2201210520FBF715FA0221684601830021817601218177BD
:208340000021C176017706A90520FBF763F901216846018381760021C17606A90520FBF7C2
:2083600059F904216846018300218176C176022141770021817706A90520FBF74BF961782E
:208380006846017002214180002141710C2181710121C1710021017160680290A06803900C
:2083A000E06804902069059069460D48F9F7ECFA0C496069086001210948F9F7EFFB0122F3
:2083C0000E210748F9F7C7FA07493720FCF7DEFA06492920FCF7DAFA002008B010BD0000F8
:2083E0000054044068000020AD8100009581000000BE00BFFEE77047014672B60820884A97
:20840000D060F120106255205060AA2090600020C043086000BF82480068C007C00F002890
:20842000F9D001207E4A10600020D060F020106262B600207047014672B61020784AD060C8
:20844000F120106255205060AA2090600020C043086000BF72480068C007C00F0028F9D0C7
:2084600001206F4A10600020D060F02010620020704770B503461D46F120694E30620024BA
:2084800015E072B6AA20664E70605520B06010782870521C6D1C62B600BF61480068C00726
:2084A000C00F0028F9D001205D4E3060641C8C42E7D3F0205A4E3062002070BDF7B5FFB0A6
:2084C000FFB089B006460F460021FFA8C161012104914802874206D9FFA8C161C0697FB05F
:2084E0007FB00CB0F0BD029600240DE002980078FFA988610298401C02908869FF2801D027
:2085000000200490601C84B2BC42EFD30498002809D0444844490860FFA83946826A30468F
:20852000FFF7A7FF6DE0750AF119681C4002814202D90120039001E000200390710A490257
:208540000191F105C90D0091039800280FD0002408E00198007805A908550198411C0191DA
:20856000601C84B2012080028442F2DB0EE0002408E00198007805A908550198411C019175
:20858000601C84B2012040028442F2DB00240DE0FFA8806A01780098001905AA1154FFA8AC
:2085A000806A411CFFA88162601C84B2BC42EFD30398002816D01B481B4908606802FFF740
:2085C0003AFF184818490860691C4802FFF733FF144815490860680205AA01218902FFF764
:2085E00048FF0EE00F48104908606802FFF723FF0C480D490860680205AA01214902FFF71E
:2086000038FFFFA8C0696AE730B50446002304E025781570641C521C5B1C8B42F8D330BDC0
:2086200000000240CDAB34127000002001020020FE0000FE000002020021FE0000FE00006A
:2086400003020022FE0000FE000004020023FE0000FE00000502040AFE0000FE00000602B9
:20866000001C020701FE00000702001DFE0000FE000008020106020702FE00000902010787
:20868000020710FE00000A02010FFE0000FE00000B02010EFE0000FE00000C020123FE0063
:2086A00000FE00000D020423FE0000FE00001002012EFE0000FE00001102012FFE0000FE0E
:2086C00000001202010F07041A07050A1302010E0704370705091402020CFE0000FE0000A0
:2086E0001502020DFE0000FE000016020319FE0000FE00000E02052BFE0000FE00000F02DB
:20870000052AFE0000FE00001704001904011B0408071804021E040301FE00001900002943
:20872000FE0000FE00001A000128FE0000FE00001B00020E070909FE00001C000318FE0087
:2087400000FE00001D00041E07090CFE00001E00051F07090BFE00002000060FFE0000FE36
:2087600000002107090AFE0000FE00002207031EFE0000FE00002307031FFE0000FE000034
:2087800000FE0000FE0000FE000001000200040008001000200040008000000100020004D9
:2087A000000800100020004000800000484A5F3735305F54465400000000000000000000E7
:2087C000000000000000000000000000484A59422D37353030544654000000000000000085
:2087E0000000000000000000000000004241543332413237394B4D363446420000000000D0
:2088000000000000000000000000000043414E5F5354445F4348305F3530304B627073009E
:208820000000000000000000000000008907000081070000DF07000000000000000000003A
:20884000963007772C610EEEBA51099919C46D078FF46A7035A563E9A395649E3288DB0EED
:20886000A4B8DC791EE9D5E088D9D2972B4CB609BD7CB17E072DB8E7911DBF906410B71D0B
:20888000F220B06A4871B9F3DE41BE847DD4DA1AEBE4DD6D51B5D4F4C785D38356986C13AB
:2088A000C0A86B647AF962FDECC9658A4F5C0114D96C0663633D0FFAF50D088DC8206E3BCC
:2088C0005E10694CE44160D5727167A2D1E4033C47D4044BFD850DD26BB50AA5FAA8B53515
:2088E0006C98B242D6C9BBDB40F9BCACE36CD832755CDF45CF0DD6DC593DD1ABAC30D926E1
:208900003A00DE518051D7C81661D0BFB5F4B42123C4B3569995BACF0FA5BDB89EB80228AA
:208920000888055FB2D90CC624E90BB1877C6F2F114C6858AB1D61C13D2D66B69041DC76CC
:208940000671DB01BC20D2982A10D5EF8985B1711FB5B606A5E4BF9F33D4B8E8A2C9077848
:2089600034F9000F8EA8099618980EE1BB0D6A7F2D3D6D08976C6491015C63E6F4516B6BFE
:2089800062616C1CD83065854E0062F2ED95066C7BA5011BC1F4088257C40FF5C6D9B065B6
:2089A00050E9B712EAB8BE8B7C88B9FCDF1DDD62492DDA15F37CD38C654CD4FB5861B24D6B
:2089C000CE51B53A7400BCA3E230BBD441A5DF4AD795D83D6DC4D1A4FBF4D6D36AE9694348
:2089E000FCD96E34468867ADD0B860DA732D0444E51D03335F4C0AAAC97C0DDD3C710550AC
:208A0000AA41022710100BBE86200CC925B56857B3856F2009D466B99FE461CE0EF9DE5E8D
:208A200098C9D9292298D0B0B4A8D7C7173DB359810DB42E3B5CBDB7AD6CBAC02083B8EDE9
:208A4000B6B3BF9A0CE2B6039AD2B1743947D5EAAF77D29D1526DB048316DC73120B63E3E3
:208A6000843B64943E6A6D0DA85A6A7A0BCF0EE49DFF099327AE000AB19E077D44930FF0AB
:208A8000D2A3088768F2011EFEC206695D5762F7CB67658071366C19E7066B6E761BD4FEB1
:208AA000E02BD3895A7ADA10CC4ADD676FDFB9F9F9EFBE8E43BEB717D58EB060E8A3D6D68A
:208AC0007E93D1A1C4C2D83852F2DF4FF167BBD16757BCA6DD06B53F4B36B248DA2B0DD8CB
:208AE0004C1B0AAFF64A0336607A0441C3EF60DF55DF67A8EF8E6E3179BE69468CB361CB1D
:208B00001A8366BCA0D26F2536E2685295770CCC03470BBBB91602222F260555BE3BBAC5B0
:208B2000280BBDB2925AB42B046AB35CA7FFD7C231CFD0B58B9ED92C1DAEDE5BB0C2649BE4
:208B400026F263EC9CA36A750A936D02A906099C3F360EEB8567077213570005824ABF95CE
:208B6000147AB8E2AE2BB17B381BB60C9B8ED2920DBED5E5B7EFDC7C21DFDB0BD4D2D386BE
:208B800042E2D4F1F8B3DD686E83DA1FCD16BE815B26B9F6E177B06F7747B718E65A0888EC
:208BA000706A0FFFCA3B06665C0B0111FF9E658F69AE62F8D3FF6B6145CF6C1678E20AA0A9
:208BC000EED20DD75483044EC2B30339612667A7F71660D04D476949DB776E3E4A6AD1AECE
:208BE000DC5AD6D9660BDF40F03BD83753AEBCA9C59EBBDE7FCFB247E9FFB5301CF2BDBDC8
:208C00008AC2BACA3093B353A6A3B4240536D0BA9306D7CD2957DE54BF67D9232E7A66B303
:208C2000B84A61C4021B685D942B6F2A37BE0BB4A18E0CC31BDF055A8DEF022D3337313052
:208C4000302D433031312D30313030433031312D56313030433031312D56313030202407D7
:208C600023312E30315F3230323430383038000056312E3332203230323430353330000050
:208C8000B08C000000000020EC02000024140000E88C000000FF0020240000003C810000DE
:208CA000E88C0000EC020020A45400004C81000001400233C01AFF011133754A09D00551EB
:208CC000890A890F09213209171E091723012D0917A0092682091750091241015303127048
:208CE0008CEAFF101901011801200649087000BF04480078802108400028F9D0012002490B
:0C8D000008707047000C02406C0000205E
:00000001FF
